:020000020000FC
:047000000C948D3E21
:047028000C94B73DD0
:10702F0012010002FF010020EB03F42F0000010208
:10703F00030109021200010100803209040000005F
:10704F00000000000C03410054004D0045004C00AF
:10705F001603410054006D00330032005500340018
:10706F004400460055000C0331002E0030002E0066
:10707F0030000403090416010C0100000C0000018C
:02708F006C7F14
:1070920012BD01BDF89A00B5089501E00895F9996D
:1070A200FECF12BD01BD20BDFA9AF99AF6CFF99929
:1070B200FECF0C944938F80104910895F8013491F7
:1070C20031962491890108950091610000930C0189
:1070D20000E80093610001E00093610005BF02E057
:1070E20005BF0C9486380091D70001600093D70049
:1070F200A89507EF04BF0091600000610093600053
:1071020000E00093600001E008950E94AA3D0E9401
:10711200B53DFDCF0CD00F7708D0006806D00061D6
:1071220004D0016028D0789408950093D80000918B
:10713200D8000895FCDF00621ED04CD009B500FFD4
:10714200FDCFF5DF0F7D17D00091E0000E7F009399
:10715200E0000091E000077F0093E0000091E20070
:1071620001600093E2000091E20008600093E200F7
:1071720078940C94743B0093D800089500910D010B
:10718200002359F40091D90000FF07C0D0DF006846
:10719200F2DF01E000930D01CDDFE0E2F2E00081D9
:1071A200018100FF0DC0008111811E7F11830083C8
:1071B20001E00093EA0000E00093EA0000931E025F
:1071C20000E00093E9000091E80003FF02C00E9482
:1071D200F23B0895A89539D000E40093600000E0E6
:1071E200009381000093800010E0009385000093DB
:1071F200840001E006BB00918100036000938100DE
:107202000091600007FFFCCF00E80093600010933C
:107212008100A89507EF04BF18D010936000209159
:1072220084003091850010938100109380001093A8
:1072320085001093840001E006BB2D3D354010F01F
:1072420002E101C002E009BD089500916000006101
:107252000093600008950E94AD3E239741D100E063
:1072620000930901B5D104811581012B51F437D165
:1072720000910701002309F4B9C000E0009307015F
:10728200B5C058D102FFFDCF37D1068335D1009367
:107292000F0132D1009310012FD1009311012CD193
:1072A2000093120129D10093130102852091130149
:1072B20030911201409111015091100116811A95DD
:1072C20041F01250A9F01A9599F11A9509F473C078
:1072D2008BC010910F01113011F411E001C010E0C8
:1072E200138799D00C3F11F414D17FC077D17DC0A0
:1072F20092D010910F01112329F01A9549F01A9595
:10730200A9F073C010E013870C3F09F06EC0ECCFF8
:1073120056D103C04CD109F468C00D911C9144D1DF
:107322000F3FC1F305E0009309015FC011E0EBCF0D
:10733200D2D029F00250E1F10A9541F056C0FDD0B9
:107342000E94A33F0FEF00930A014FC0552319F08B
:107352005A9579F04AC04ED00DEF04BF74D0EAD0EE
:1073620003FFFDCF67D051D04AD008E00093600000
:10737200FFCF40D068D0DED003FFFDCF5BD03FD03F
:1073820044D00FEF1FE004C009811A810150104060
:1073920009831A8309811A81012BB1F700E800934E
:1073A200610000910C01009361000C940000FFCF7A
:1073B20001E003871AC08FD019F00A9539F015C081
:1073C200535098F4BAD002E000870FC0505339F0FE
:1073D2005A9541F05F52B1F35A95A1F306C002E00B
:1073E2000883F0CF01E0FCCFA8D079D02396E4E067
:1073F2000C94BA3E01E005BF00E005BF089500917C
:10740200D8000F770093D800089509B50D7F09BD04
:1074120000E009BD08955183408333832283109194
:10742200E8001B7F1093E8001091E8001F7710938B
:10743200E80008955DD053D0F8940091E000016017
:107442000093E000089579D04AC0219749D0009175
:107452000601035019F00250B9F00BC03CD021F0E4
:107462000A9559F00A9529F400910A010C3F19F482
:1074720050D02196089567D0FCCF0091010100936E
:10748200F100009100010AC01091100124D019F0FE
:107492000A9549F0EECF135018F400E00093F10082
:1074A2001ED044D0E6CF105339F01A9539F01F524E
:1074B20041F01A9541F0F4CF08E5F0CF00E006D094
:1074C200EDCF02E0FCCF04E001D0E8CF10E020E0F5
:1074D20030E00C94113F00910F010023089521C068
:1074E2000BD008D007D00093040106D00093050109
:1074F20021D00BC000D008830091F10008950091C3
:10750200EB0000620093EB0015D0077F0093E800C8
:107512000895F5DF02E00093080103E000930901FA
:10752200089559D007D000FFFDCF089503D002FF80
:10753200FDCF03C00091E8000895FCDF0B7FE6DF7A
:10754200F9DF0F77E3CF0E94AC3E42D038D006C0BD
:107552002BD00093F1002BD059F43DD0082F092BEA
:10756200A9F0E8DF02FD12C0E5DF00FFFDCF4424F1
:10757200042D4394003289F300910B0100230D91F5
:107582001C9131F311970E945838E3CFD3DF00FFEB
:10759200FDCF21D0CFDF00FFFDCFCCDF02FFFDCF3B
:1075A200CCDFE5E00C94B93E11970C945C380D9158
:1075B2001C910F5F1F4F1C930E93019708958281B8
:1075C200938100811181801B910B0196DF01089547
:1075D200E0E0F1E00895AEDF0E7F98CF0E94A93E71
:1075E200F7DF80819181A081B181AF710481158122
:1075F20000521040048315830AC000910B0100233E
:1076020031F4A301920103E911E00E943B3F47D00C
:10761200B8F1662477242C0111C06EDFF301ED5618
:10762200FE4F008301E0600E00E0701E01960091A3
:10763200F200002311F033D0B8F47FDF30D0E8F24B
:10764200F301B096E238F040C0F674DF02FFFDCFDE
:107652000091F200BDDF24813581201B304024835C
:107662003583E5CF49DFAA95AA23E1F700910B0103
:10767200013099F62091F1008C010E945038D6CF4A
:1076820004811581012B21F055DF02FFFDCF55DF6B
:10769200A2DF50DF00FFFDCFE8E00C94B63EE0E051
:1076A200F1E0028113810817190708952091EB0078
:1076B20021602093EB000093EC000091ED0002703A
:1076C200012B0093ED000091ED0002600093ED00AC
:1076D2001091EE00012F000F00E0001F0895412FCE
:1076E2000093E900089500E009D000FD05C000E024
:1076F200F7DF10E202E0DACF00E00895F1DF009157
:10770200EB0008950F770132A9F5112369F11A955B
:1077120059F01A9561F01A9569F01A95F9F01A95CF
:10772200C1F01A95D9F024C00E942C3920C00E94C1
:10773200263A1DC029D00091090123D001E01FD0B3
:1077420020D0009108011BD00E94923A0E94973AE1
:107752000EC01AD00091080114D007C002E00093B5
:10776200080100E0009309010FD00E94923A03C081
:107772000E94803A02C001E0089500E0089501D01D
:1077820000E00093F10008950091E800077F009364
:10779200E800089508950350F9F4112339F01A9579
:1077A20051F01A9581F01A9599F016C004E016D09E
:1077B20001E810E703C011D003E510E7E7E1F2E0CA
:1077C20000831183D8CF06E109D00FE510E7F6CF89
:1077D20004D005E710E7F2CFD0CF0CE000931A02F5
:1077E200089527D120D100931D02E1D0212F11232A
:1077F20029F12A95E9F02250F1F0225099F02A95C8
:1078020049F0225061F02A9581F02A95E1F02A95FB
:10781200E9F023C0003809F44FC00C94833B0038D0
:10782200E1F7C8C00023C9F71EC00023B1F72DC07D
:10783200033098F744C1033080F70BC1003868F376
:10784200033858F7C9C0013841F77BC1013051F400
:10785200FCD0BFD000FD06C0FCCF0E94833B0023BA
:1078620009F41ED008951091E3001078DCD00F7750
:10787200012B0093E300E9D0ACD000FFFDCF0091D3
:10788200E30000680093E300089591D0123040F4C1
:107892000FD010931E02DAD000911E020C94CB3B43
:1078A2000091EB0001D004C000620093EB00089548
:1078B2000091E800077FC0C0BA93AA93229700E024
:1078C2000093190274D0AFD0202F2A9519F02A956F
:1078D200E9F022C002E100931A020FE210E7E7E1A9
:1078E200F2E0008311839DD008839DD00983E0DFFD
:1078F20000911A0210E02881398102171307A8F4B7
:107902000F7181F401E00093190211C002E10093AA
:107912001A0201E410E7E3CF0E94CC3B002319F7DF
:107922008ED040C01093190202C020931A027ED05A
:10793200A7E1B2E001C08AD000911A02002309F146
:1079420048D004FD1EC045D000FD03C042D004FF54
:10795200FACF10E0012F1395003281F0ED91FC91E6
:107962001197049133D02D913C912F5F3F4F3C935F
:107972002E93FD0103810A95038361F72AD004FF48
:10798200DACF00911902013039F423D004FD04C08A
:1079920020D000FFFDCF5AD01CD004FFFDCF46D02F
:1079A20018D00B7F49D02296A991B99108951091D0
:1079B200F10008957DDF00911E0208D047D009D062
:1079C2000F773AD006D002FFFDCFBFC00093F1007F
:1079D20008950091E800089524D010911D021058D6
:1079E20029F01A9589F01A9591F019C061DF00917A
:1079F2001C02ECDF00E0EADF29D0EBDF02FFFDCF63
:107A020018D0E7DF0F770CC053DF00E0F2CF51D080
:107A12000F7710E0F801E55EFD4F0081EACF0FD04D
:107A22000BC001D000D00091F1000895D2DF0F7E8B
:107A320003C00091E8000B7F0093E80008950091D5
:107A4200EB0032DFC6DF077F089532DFC2DF0E7F31
:107A5200F3CF00911D02002329F00A9509F10A953E
:107A620031F01EC0E0DF0A9561D0D9F41AC061D0AE
:107A7200B9F4D9DF0F7711F416D01BD00093E900C7
:107A82001091EB0010FF0BC00ED010E01093E90034
:107A920021E0F801E55EFD4F20834FD003C042D0C4
:107AA20045D0CFDFC9CF1091EB0010621093EB00ED
:107AB20008951091E800177F1093E800089500914F
:107AC2001D02002311F4AFDF02C0013011F4B7DF51
:107AD200B3CF023031F52DD019F52091F1002F7777
:107AE2002093E90023D000FF19C081F01FD000616C
:107AF200DCDE01E010E0422F0E949F3E0093EA008C
:107B020000E00093EA0012D00860CFDE0BD030E034
:107B1200F901E55EFD4F008310D0DACF03D0D7CF55
:107B2200BFDE089500E00093E90008950091EB00A4
:107B3200089579DF3CDF00230895BADE4ADF0E7F25
:107B4200089583DF46DF02FFFDCF73DF42DF0F7749
:107B520073CF0091D70001600093D7000E948B3849
:107B620000E000931F0208950C94BF388A93FA93A1
:107B7200EA933A922A921A920A927A936A935A93BF
:107B82004A933A932A931A930A938FB70091DA0091
:107B920000FF24C00091D80000FF20C00EEF009328
:107BA200DA000091D90000FF11C001E000930D013D
:107BB200ABD0026096D09AD00860A2D00E949B38C7
:107BC2000091E0000E7F0093E00008C000E0009307
:107BD2000D0100931E0298D0046083D07FD002FF73
:107BE20005C084D002FF02C00BEF75D077D000FF32
:107BF2001BC07CD000FF18C001E000930E016AD0C8
:107C020083D000626ED00EEF6FD0006179D06ED05B
:107C12000F7D76D00091D80000620093D80009B59C
:107C22000D7F09BD00E009BD59D004FF20C05ED020
:107C320004FF1DC009B500FD05C00E94EB3809B55F
:107C420000FFFDCF0091D8000F7D0093D80042D0F5
:107C520000910E01002359F04CD00FEE45D00F7E5B
:107C620052D000643ED042D001604AD042D036D0D9
:107C720005FF0FC03BD005FF0CC000E000930E01D2
:107C820035D00F7E3DD00FED2FD00F7D3CD0006858
:107C920028D024D003FF0DC029D003FF0AC000E082
:107CA20000931F0207EF17D00E94743B2DD0116082
:107CB20018D08FBF09911991299139914991599100
:107CC200699179910990199029903990E991F991E6
:107CD200899118950FEE0093E10008950091E1005B
:107CE20008951183008308950093E1000091E2005A
:107CF20008950091E200006203D00091E200086062
:107D02000093E2000895FCDFE0E2F2E000811181DD
:107D1200089500008895FECF01E60DBF02E00EBF78
:107D2200C2EED2E00E947438002311F00E94D33ECA
:107D32000E9465380E948A3E0C948A3E4A951AF047
:107D4200000F111FFBCF0895BA92AA929A928A92BB
:107D52007A926A925A924A92BA93AA939A938A937D
:107D62000895BB84AA84998488847F806E805D8014
:107D72004C80BB81AA8199818881F0E00FB6F8948A
:107D8200CE0FDF1F0FBE089520E006D0E9F7089559
:107D9200259102D0E9F708952D9301501040202F2C
:107DA200212B089585E890E7FC0105911491FC01CF
:107DB2003296A591B491FC01349625913491422FCB
:107DC200432B19F0F901E4DF01C0DEDF069610E76C
:107DD2008139910748F308952F930CD02F9101D048
:107DE20008953CD0F12FE02F45E047BFE89536D00B
:107DF20012D0089533D0F12FE02F43E047BFE8952A
:107E02002DD008952BD0F12FE02F43E047BFE89506
:107E120025D001D0089522D041E147BFE8951EC088
:107E22001DD0F12FE02F41E247BFC895002D16C0AB
:107E320015D0F12FE02F49E047BFC895002D0EC0A5
:107E4200F32FE22F012E102E41E047BFE89506C026
:107E520005D0002E29E027BFE89500C0022E27B7E3
:107E620020FDFCCF202D0895022E27B726FDFCCF42
:107E7200202D08950E94A53E22974801C901DA01EA
:107E820010C05BD001E0A00E00E0B01E00E4A0161E
:107E920000E0B00608F440C0830120E030E00E9418
:107EA200F23E0A2F0B2B09F440C0082F0F7710E087
:107EB2002C01401A510A320100E4A02E03C00A2FFD
:107EC2000B2BE1F04816590680F0F40101914F01A5
:107ED2000983119729F001914F010883119711C06D
:107EE200F2013196049108830CC0F20104910983D6
:107EF2003196E817F907A1F7F401EDCF1BD00883FB
:107F020019839201088119810E94213F16D0AA94F7
:107F1200B1F62301AA24BB240DD0312F0F3F3F4FCE
:107F220009F4AFCF83011DD0B7CF01E02296ECE078
:107F32000C94B23E82010C945F3802E0400E00E0E5
:107F4200501E08959A938A9380E090E08C0109D0A4
:107F520080589F4F8F3F0FE69007C0F38991999108
:107F6200089520E030E00C94FB3E00000000000089
:067F720000000000FC000D
:107FE4000C94ED3E0C94113F0C94193F0C94213FDA
:0C7FF4000C94F23E0C94033F0C94293FC7
:040000030000700089
:100000000C947C050C94C0050C94C0050C94C005A0
:100010000C94C0050C94C0050C94C0050C94C0054C
:100020000C94C0050C94C0050C94C7180C94991935
:100030000C94B2270C94C0050C94C0050C94C00518
:100040000C94C0050C94C0050C94C0050C94C0051C
:100050000C94C0050C941A280C94C0050C94C0058F
:100060000C94C0050C94C0050C94C0050C94C005FC
:100070000C94C0050C94C0050C94C0050C94C005EC
:100080000C94E50E0C94C0050C94C0050C94C005AE
:100090000C94C0050C94C0050C94C0050C94C005CC
:1000A0000C94C0050C94C0050C94C0051B062B06CF
:1000B0003D064D06530662066E06730680068806E8
:1000C00098069D06061A281A161B281A161B6D1A62
:1000D000901A161BE51AF81AFB1DFB1D381E381E58
:1000E000921ED01E48214821E91E4821EA1FEA1F1E
:1000F000AD20C4204821332107634236B79BD8A7DF
:100100001A39685618AEBAAB558C1D3CB7CC57633C
:10011000BD6DEDFD753EF6177231BF000000803FEA
:1001200008000000BE922449123EABAAAA2ABECD06
:10013000CCCC4C3E00000080BEABAAAAAA3E000078
:100140000000BF000000803F000000000008417870
:10015000D3BB4387D1133D190E3CC3BD4282AD2BA7
:100160003E68EC8276BED98FE1A93E4C80EFFFBE9F
:1001700001C4FF7F3F000000000035001E001F008B
:100180002000210022002300240025002600270053
:100190002A002B0014001A000800150017001C008C
:1001A00018000C00120013004C0029000400160077
:1001B000070009000A000B000D000E000F003300BD
:1001C0003400E1001D001B000600190005001100AD
:1001D000100036003700380028000530E000E2004B
:1001E000E30003302C002C0004305000510052007A
:1001F0004F0035001E001F002000210022002300B8
:1002000024002500260027002A002B0014001A00D5
:10021000090013000A000D000F0018001C00330035
:100220004C002900040015001600170007000B0001
:10023000110008000C0012003400E1001D001B003A
:100240000600190005000E001000360037003800C7
:1002500028000530E000E200E30003302C002C0011
:1002600004305000510052004F0035001E001F00A6
:100270002000210022002300240025002600270062
:100280002A002B0034003600370013001C00090040
:100290000A00060015000F004C002900040012009F
:1002A000080018000C0007000B00170011001600D2
:1002B0003800E100330014000D000E001B000500A3
:1002C00010001A0019001D0028000530E000E200AF
:1002D000E30003302C002C00043050005100520089
:1002E0004F0035021E021F022002210222022302B9
:1002F00024022502260227022A0035021E021F02BE
:1003000020022102220223022402250226022702C1
:100310004C004C003A003B003C003D003E003F00DA
:100320002D022E022F023002310201004000410056
:1003300042004300440045000100010001000100AB
:1003400001000100010001000100010001000100A5
:100350000100AB00AA00A900AE0035001E001F007E
:100360002000210022002300240025002600270071
:100370002A0035001E001F0020002100220023005B
:1003800024002500260027004C004C003A003B00CA
:100390003C003D003E003F002D002E002F003000AD
:1003A000310001004000410042004300440045008C
:1003B0000100010001000100010001000100010035
:1003C00001000100010001000100AB00AA00A9002A
:1003D000AE0000000000000000000000000000006F
:1003E000000000000000000000000000000000000D
:1003F00000000000000000000000000000000000FD
:1004000000000000000000000000000000000000EC
:1004100000000000000000000000000000000000DC
:1004200000000000000000000000000000000000CC
:100430000000000000000000000003300000000089
:100440000430000000000000000000000000000078
:10045000000000000000000000000000000000009C
:10046000000000000000000000000000000000008C
:10047000000000000000000000000000000000007C
:10048000000000000000000000000000000000006C
:1008F000000000000000000000003A003B003C0047
:100900003D003E003F0040004100420043004400E3
:10091000450001000050010001000100010001003C
:1009200001000100010001004C0001000100010074
:1009300007300630135012500030013002300100F1
:10094000010001000B300A300930083001000100BD
:10095000010001000100010001000100010001008F
:10096000010001000100010001000100010001007F
:1009700001002A0354006800650020005000720046
:1009800065006F006E006900630020004B00650089
:10099000790062006F0061007200640000002C03A7
:1009A0004F007200740068006F006C0069006E00F8
:1009B00065006100720020004B0065007900620054
:1009C0006F006100720064007300000004030904FA
:1009D00009025400030100A0FA0904000001030108
:1009E0000100092111010001223F000705810308D0
:1009F000000A09040100010301020009211101009C
:100A000001224D000705820308000A0904020001C3
:100A100003000000092111010001223600070583AF
:100A20000308000A1201100100000008EDFE6160D9
:100A300001000102000105010980A10185021601E2
:100A40000026B7001A01002AB70075109501810031
:100A5000C0050C0901A1018503160100269C021A9C
:100A600001002A9C02751095018100C00501090250
:100A7000A1010901A1000509190129051500250198
:100A80009505750181029501750381010501093004
:100A900009311581257F9502750881060938158170
:100AA000257F950175088106050C0A3802158125F8
:100AB0007F950175088106C0C005010906A10105E1
:100AC0000719E029E71500250195087501810295B0
:100AD0000175088101050819012905950575019120
:100AE000029501750391010507190029FF150025DD
:100AF000FF950675088100C011241FBECFEFDAE014
:100B0000DEBFCDBF04B603FE24C08091F3039091F5
:100B1000F403A091F503B091F6038730904BA74002
:100B2000B04BB9F41092F3031092F4031092F50352
:100B30001092F60314BE84B7877F84BF88E10FB696
:100B4000F89480936000109260000FBEE0E0F8E33C
:100B5000099512E0A0E0B1E0E8EAF3E602C00590F2
:100B60000D92A63FB107D9F713E0A6EFB2E001C09E
:100B70001D92A33FB107E1F70E940D160C94D231EC
:100B80000C940000279A2F988FEF9FEF9093870087
:100B9000809386008AE08093800089E180938100C1
:100BA0000C94092D282F81110BC080918000877F24
:100BB0008093800010928D0010928C002F980895E1
:100BC0002F9880918000886080938000233019F4F2
:100BD0008FEF9FEF0FC083E090E0821B9109880F99
:100BE000991F2FEF3FEFA90102C0569547958A95AF
:100BF000E2F7CA0190938D0080938C000895CF9303
:100C0000DF93EC010E94AE28BE0180E090E0DF910E
:100C1000CF910C9428250F931F93462F50E04C3012
:100C2000510508F098C0DC01FA01EA5AFF4F12960C
:100C30008C910C949631882309F48DC000E010E06B
:100C4000980140E064E070E089EC91E00E9463125A
:100C500081E090E00FC0882309F47DC000E010E03F
:100C6000980140E066E070E089E591E00E9463123F
:100C700082E090E00E94FF056EC0882309F46BC0FB
:100C800000E010E0980140E068E070E089E891E061
:100C90000E94631284E090E0EDCF882311F083E09E
:100CA00005C083E00CC0882349F084E00E94A5259C
:100CB00040E164E083E00E94C90A4DC084E00E94E4
:100CC000C625F6CF882331F085EE0E948F1C0E9446
:100CD000602D41C085EE0E94571D3DC08823D9F18B
:100CE0000E94F70D38C08823B1F10E94F00D00E09A
:100CF00010E0980140E064E070E089EE91E029C0E6
:100D0000882349F185E00E94C6250E94180E23C061
:100D1000882309F100E010E0980140E068E070E00D
:100D200089E191E00E94631285E00E94A52513C02D
:100D3000882389F00E94F61204C0882361F00E9483
:100D4000011300E010E0980140E068E070E089E104
:100D500091E00E94631280E090E01F910F9108954E
:100D60000F931F932FEF89EF90E021508040904028
:100D7000E1F700C0000000E010E0980140E064E00E
:100D800070E089EE91E00E9463121F910F91089527
:100D9000CF92DF92EF92FF920F931F93CF93DF9347
:100DA000CDB7DEB7CC58D1090FB6F894DEBF0FBE71
:100DB000CDBF2091B30325FFC5C08C01FC019281FA
:100DC00080910001992309F460C096E4E5E2F2E025
:100DD000DE01A95BBF4F01900D929A95E1F7F801F2
:100DE0009081E091F602F091F702E90FF11DEE0F0C
:100DF000FF1F27E430E02C0F3D1FE20FF31F60813F
:100E00007181680F711D882777FD8095982F0E944A
:100E1000A42E20E030E040E451E40E94092E6B0152
:100E20007C01F801218185E090E0821B9109BC01E1
:100E3000882777FD8095982F0E94A42E9B01AC01F6
:100E4000C701B6010E94A12D9B01AC0160E070E0DA
:100E500080E090E40E94173020E030E04CE551E45F
:100E60000E94B42F4FE050E0C457DF4F0FB6F89404
:100E7000DEBF0FBECDBFDF91CF911F910F91FF90CD
:100E8000EF90DF90CF900C94031296E4E5E2F2E04D
:100E9000DE01119601900D929A95E1F7F80190818B
:100EA000E091F602F091F702E90FF11DEE0FFF1F3E
:100EB00021E030E02C0F3D1FE20FF31F60817181B4
:100EC000680F711D882777FD8095982F0E94A42EAA
:100ED00020E030E040E451E40E94092E6B017C01E7
:100EE000F801218185E090E0821B9109BC018827EF
:100EF00077FD8095982F0E94A42E9B01AC01C7011D
:100F0000B6010E94A12D9B01AC0160E070E080E081
:100F100090E40E94173020E030E04CE551E40E945C
:100F2000B42FC457DF4F0FB6F894DEBF0FBECDBF4E
:100F3000DF91CF911F910F91FF90EF90DF90CF90B5
:100F40000C944B0EC457DF4F0FB6F894DEBF0FBEA4
:100F5000CDBFDF91CF911F910F91FF90EF90DF9068
:100F6000CF9008950F931F9300E010E0980140E0A8
:100F700063E070E081E091E00E9463122FEF82E570
:100F800097E0215080409040E1F700C000001F91A1
:100F90000F91089508950E94C2056E9A769A0C9456
:100FA000B0060C94CA070C94C8060895880F991FC0
:100FB000FC01E650F040859194910895880F991FA7
:100FC000FC01E658FE4F8591949108950F931F936D
:100FD000CF93DF93EC01811520E49207A0F5C115B2
:100FE00080E3D80708F0E1C0C83ED105D8F4C03E80
:100FF000D10508F0EEC1C83AD10578F4C53AD1055B
:1010000008F074C0C130D10509F46DC008F4DEC128
:10101000C430D10508F0DDC1D9C1CB3BD10508F4FE
:1010200070C0D4C1C11590E2D90708F0B9C0C1158C
:1010300021E0D20708F0CDC1C03FD10508F4C6C1F8
:101040008E01106506C2C13080E5D80709F4BDC025
:1010500068F5C13120E4D20709F4AEC050F4C031C4
:1010600090E4D90708F0A5C0CF70DD278E01146D7C
:10107000F0C1C33120E4D20709F4A4C008F49FC032
:10108000C115D04509F0A2C10E946C210E94180E22
:101090000E94B2079FEF24E38CE0915020408040F3
:1010A000E1F700C000000E943F28D3C1C11520E62F
:1010B000D20730F4C11581E5D80708F48CC02DC1E2
:1010C000C11590E7D90708F481C1C11520E8D207FE
:1010D00008F478C1C11580E9D80708F077C1DF703E
:1010E0008E01106AB6C101E010E0B3C1C53AD10566
:1010F00009F471C1C63AD10509F070C102E810E4E3
:10110000A8C1C83AD10509F46CC1C93AD10509F49E
:101110006BC1CA3AD10509F46AC1CB3AD10509F4C9
:1011200069C1CC3AD10509F468C1CD3AD10509F4B9
:1011300067C1C03BD10509F466C1CE3AD10509F4B7
:1011400065C1CF3AD10509F464C1C13BD10509F4A9
:1011500063C1C23BD10509F462C1C33BD10509F4A7
:1011600061C1C43BD10509F460C1C53BD10509F497
:101170005FC1C63BD10509F45EC1C73BD10509F487
:101180005DC1C83BD10509F45CC1C93BD10509F477
:101190005BC1CA3BD10509F45AC100E014E459C14E
:1011A000CE019F700E94DE0755C1DD278E01106CB5
:1011B00050C100E011ED4DC100E010ED4AC100E06A
:1011C00012ED47C100E013ED44C18091C703816077
:1011D0008093C7033EC10E949B28811102C00E94D8
:1011E00077280E94B32890E09093F2038093F10354
:1011F000C23090E5D90721F48091F103816086C067
:10120000C43020E5D20721F48091F10382607EC0D2
:10121000C63080E5D80721F48091F103846076C060
:10122000C83090E5D90719F48091F10327C0CA307E
:1012300020E5D20721F48091F103806167C0CC30B2
:1012400080E5D80721F48091F10380625FC0CE3041
:1012500090E5D90721F48091F103806457C0C03133
:1012600020E5D20721F48091F10380684FC0C2319C
:1012700080E5D80729F48091F1038460886046C036
:10128000C33090E5D90721F48091F1038E7F3EC0F1
:10129000C53020E5D20721F48091F1038D7F36C05F
:1012A000C73080E5D80721F48091F1038B7F2EC0F1
:1012B000C93090E5D90719F48091F10326C0CB30ED
:1012C00020E5D20721F48091F1038F7E1FC0CD303D
:1012D00080E5D80721F48091F1038F7D17C0CF30CE
:1012E00090E5D90721F48091F1038F7B0FC0C131C4
:1012F00020E5D20721F48091F1038F7707C0C33135
:10130000D04531F48091F1038B7F877F8093F10387
:101310008091F1030E94B7289CC08D2F99278F7070
:10132000992781309105D9F49E012370332702C09B
:10133000880F991F2A95E2F79C688E0144E0000F00
:10134000111F4A95E1F700271370802B912B53E072
:10135000CC0FDD1F5A95E1F7C076DD272FC0823014
:10136000910531F4DC2FCC278E01016F106A71C01A
:101370008330910569F4CE018370992701E010E074
:1013800002C0000F111F8A95E2F7C8019C680FC0C8
:10139000049709F05EC0CE018370992701E010E048
:1013A00002C0000F111F8A95E2F7C8019A6823E076
:1013B000CC0FDD1F2A95E1F7C07ED7708C010C2B76
:1013C0001D2B47C0DF708E01106243C000E010E0AB
:1013D00040C08E013EC001E810E43BC003E810E4C9
:1013E00038C002EE14E435C009EE14E432C00AEE4F
:1013F00014E42FC005EB14E42CC006EB14E429C060
:1014000007EB14E426C00CEC14E423C00DEC14E448
:1014100020C003E815E41DC00AE815E41AC002E97B
:1014200015E417C004E915E414C001E216E411C084
:1014300003E216E40EC004E216E40BC005E216E473
:1014400008C006E216E405C007E216E402C00AE29C
:1014500016E4C801DF91CF911F910F9108959CE090
:10146000799FF00111249CE3899FE00DF11D112467
:10147000E60FF11DEE0FFF1FE658FE4F8591949188
:10148000803E9105E0F4803C910558F5813391054B
:1014900009F46FC048F48932910509F463C08A32B7
:1014A000910509F46DC072C089339105E9F0823865
:1014B0009105D1F08533910509F44DC067C0833E95
:1014C000910581F138F4803E9105B9F0823E910595
:1014D000D9F05CC0863E910561F1873E9105A1F18E
:1014E00055C00E94D60708952091F10320FD02C047
:1014F00021FF4CC080EE90E049C08091F10380FF55
:10150000F9CF89E390E042C08091F10382FF0EC0E1
:101510008091F10384FF03C080E090E037C083EE48
:1015200090E034C08091F10382FFF2CF82EE90E030
:101530002DC08091F10383FF0BC08091F10384FDE6
:10154000EBCF87EE90E022C08091F10383FFF5CFCF
:1015500086EE90E01BC08091F10385FF07C089E211
:1015600090E014C08091F10385FFF9CF85E390E00E
:101570000DC08091F10386FF07C08AE290E006C0AB
:101580008091F10386FFF9CF81E390E00E94E607A6
:101590000895CF92DF92EF92FF920F931F9301E095
:1015A00010E020E030E06801790104C0CC0CDD1CC3
:1015B000EE1CFF1C8A95D2F704C0000F111F221FDA
:1015C000331F6A95D2F70C291D292E293F29C09077
:1015D000B303D090B403E090B503F090B603C022FB
:1015E000D122E222F322842FC016D106E206F306AE
:1015F00041F41F910F91FF90EF90DF90CF900C94EA
:10160000A5251F910F91FF90EF90DF90CF900C9444
:10161000C62508950C94090B5F926F927F928F926A
:101620009F92AF92BF92CF92DF92EF92FF920F9371
:101630001F93CF93DF93CDB7DEB72A970FB6F894F9
:10164000DEBF0FBECDBFCE0101966C014E019BE007
:10165000890E911C20E030E040E050E060E070E056
:1016600000E010E0E12CF12C6C2C5D2C8AE0782E4F
:10167000AA24A394B12CEBE6F2E0A62DB52D872D7C
:1016800001900D928A95E1F7F601819191916F0198
:10169000FC01E07FFF27E032F10559F48F709927B4
:1016A000F50102C0EE0FFF1F8A95E2F7EE2AFF2A2E
:1016B00037C0E033F10559F48F709927F50102C066
:1016C000EE0FFF1F8A95E2F70E2B1F2B29C0E03487
:1016D000F10559F48F709927F50102C0EE0FFF1F35
:1016E0008A95E2F76E2B7F2B1BC0E035F10559F48C
:1016F0008F709927F50102C0EE0FFF1F8A95E2F760
:101700004E2B5F2B0DC0E036F10551F48F709927F9
:10171000F50102C0EE0FFF1F8A95E2F72E2B3F2B3B
:10172000C814D90409F0A7CF84B19E2D90958923C0
:1017300084B985B1E82AE5B887B1902F90958923BF
:1017400087B988B1082B08B98AB1962F909589235B
:101750008AB98BB1682B6BB98DB1942F9095892381
:101760008DB98EB1482B4EB980B3922F90958923B5
:1017700080BB81B3282B21BB2A960FB6F894DEBF1D
:101780000FBECDBFDF91CF911F910F91FF90EF90D2
:10179000DF90CF90BF90AF909F908F907F906F9091
:1017A0005F9008955F926F927F928F929F92AF9217
:1017B000BF92CF92DF92EF92FF920F931F93CF933E
:1017C000DF93CDB7DEB768970FB6F894DEBF0FBED4
:1017D000CDBF85B7806885BF85B7806885BF0E940B
:1017E0000C0BCE0101966C014E0199E1890E911C02
:1017F00020E030E040E050E060E070E000E010E029
:10180000E12CF12C6C2C5D2C88E1782EAA24A39479
:10181000B12CE5E7F2E0A62DB52D872D01900D92B4
:101820008A95E1F7F601819191916F01FC01E07FCA
:10183000FF27E032F10559F48F709927F50102C0B6
:10184000EE0FFF1F8A95E2F7EE2AFF2A37C0E0333A
:10185000F10559F48F709927F50102C0EE0FFF1FB3
:101860008A95E2F70E2B1F2B29C0E034F10559F4BD
:101870008F709927F50102C0EE0FFF1F8A95E2F7DE
:101880006E2B7F2B1BC0E035F10559F48F70992723
:10189000F50102C0EE0FFF1F8A95E2F74E2B5F2B7A
:1018A0000DC0E036F10551F48F709927F50102C0A3
:1018B000EE0FFF1F8A95E2F72E2B3F2BC814D90499
:1018C00009F0A7CF84B19E2D9095892384B985B165
:1018D000E82AE5B887B1902F9095892387B988B118
:1018E000082B08B98AB1962F909589238AB98BB1B4
:1018F000682B6BB98DB1942F909589238DB98EB1DA
:10190000482B4EB980B3922F9095892380BB81B329
:10191000282B21BBE2E0F3E0A8EFB2E01192119294
:101920001D921D9283E0EC30F807C1F768960FB660
:10193000F894DEBF0FBECDBFDF91CF911F910F9105
:10194000FF90EF90DF90CF90BF90AF909F908F90DF
:101950007F906F905F900C94CB075F926F927F9215
:101960008F929F92AF92BF92CF92DF92EF92FF92AF
:101970000F931F93CF93DF93CDB7DEB7A2970FB628
:10198000F894DEBF0FBECDBF6E0149E1C40ED11C7D
:1019900088EFA82E82E0B82E75019AE0592E4601F4
:1019A00001E010E028E1622E35E0732EEBE6F2E074
:1019B000D401852D01900D928A95E1F7D6018D9184
:1019C0009D916D019C01207F33272032310591F4D8
:1019D00024B18F709927F80102C0EE0FFF1F8A957E
:1019E000E2F7CF01922F982B94B995B18095892376
:1019F00085B953C02033310591F427B18F709927F1
:101A0000A80102C0440F551F8A95E2F7CA01922F20
:101A1000982B97B998B18095892388B93EC0203416
:101A2000310591F42AB18F709927D80102C0AA0F0D
:101A3000BB1F8A95E2F7CD01922F982B9AB99BB1E3
:101A4000809589238BB929C02035310591F42DB1BA
:101A50008F709927F80102C0EE0FFF1F8A95E2F7F9
:101A6000CF01922F982B9DB99EB1809589238EB975
:101A700014C02036310589F420B38F709927A8014E
:101A800002C0440F551F8A95E2F7CA01922F982B86
:101A900090BB91B38095892381BB50EA5A95F1F7A9
:101AA000BE016F5F7F4F20E030E040E050E0E5E7AF
:101AB000F2E0DE011196862D01900D928A95E1F7F4
:101AC000DB018D919D91BD01FC01E07FFF27E0329C
:101AD000F10511F4E3B113C0E033F10511F4E6B1FF
:101AE0000EC0E034F10511F4E9B109C0E035F105AB
:101AF00011F4ECB104C0E036F105B9F4EFB1F0E057
:101B00008F70992702C0F595E7958A95E2F7E0FD79
:101B100008C0C801042E02C0880F991F0A94E2F77A
:101B200002C080E090E0282B392B4F5F5F4F4C3094
:101B3000510509F0BCCFF70180819181821793078D
:101B400021F031832083709209020E940C0BF2E095
:101B5000EF0EF11C42E0E41643E0F40609F026CF54
:101B6000809109028823C9F081508093090288235B
:101B700039F08FE99FE00197F1F700C000000DC038
:101B8000E2E0F3E0D5018D919D915D018193919308
:101B9000B2E0AB16B3E0BB06A9F70E94D10781E023
:101BA000A2960FB6F894DEBF0FBECDBFDF91CF91E6
:101BB0001F910F91FF90EF90DF90CF90BF90AF906B
:101BC0009F908F907F906F905F900895E82FF0E046
:101BD000EE0FFF1FEE5FFC4F808191810895089505
:101BE0008091DC0381608093DC030C94C928809190
:101BF000DC038E7F8093DC030C94C9280E949B2811
:101C0000811102C00E9477280E94C5288093DC03BE
:101C10003E9A809171008D7F8093710082E0809365
:101C200090008AE18093910081E080930E030895F3
:101C300080910E03811102C00E94FE0D10925E037E
:101C400010925D03809171008D7F8093710080916F
:101C500090008F77809390001092200310921F03C2
:101C600010925703109258031092590310925A037E
:101C70001092560310925503E5E3F3E0A5E2B3E0BA
:101C800011921192119211921D921D9283E0E535ED
:101C9000F807B1F70895CF92DF92EF92FF920F937A
:101CA0001F93CF93DF9320911F03222309F484C055
:101CB0006B017C0180910E03811102C00E94FE0D18
:101CC00005E513E0C7E0D0E0A7019601F801929185
:101CD0008291729162918F010E94052E811131C013
:101CE000FE01EE0FFF1FEE0FFF1FEB5CFC4F10829B
:101CF000118212821382DE01AA0FBB1FAB5DBC4FA3
:101D000011961C921E92C730D105E9F021964481AC
:101D10005581668177814083518362837383148206
:101D200015821682178212968D919C9113971196A7
:101D30009C938E9313961C921E9212973496129631
:101D4000E2CF219708F680915D0390915E030197A1
:101D500097FD05C090935E0380935D0304C01092CD
:101D60005E0310925D0380915D0390915E0320916C
:101D70005B0330915C032817390724F010925C0351
:101D800010925B03892BC1F4809171008D7F809349
:101D90007100809190008F7780939000109257038C
:101DA000109258031092590310925A03109256033E
:101DB0001092550310921F03DF91CF911F910F9145
:101DC000FF90EF90DF90CF9008951F920F920FB683
:101DD0000F9211244F925F926F927F928F929F92F7
:101DE000AF92BF92CF92DF92EF92FF922F933F93E9
:101DF0004F935F936F937F938F939F93AF93BF9313
:101E0000CF93DF93EF93FF9380911F03882309F40F
:101E10009BC1C0915D03D0915E031C161D060CF0A2
:101E200093C140900F035090100360901103709085
:101E3000120320E030E0A901C301B2010E94B02FDB
:101E400018160CF065C0C130D10509F452C080915C
:101E50005B0390915C03BE010E9482317C019093F0
:101E60005C0380935B038090210390902203A090F9
:101E70002303B090240320E030E040E85FE3C50195
:101E8000B4010E94A12D60932103709322038093DB
:101E9000230390932403F701EE0FFF1FEE0FFF1FA4
:101EA000EB5CFC4FA301920160817181828193817F
:101EB0000E94092E20E030E040E05EE30E94B42F53
:101EC0009B01AC01C501B4010E94B02F18168CF41F
:101ED000C7010196BE010E94823190935C038093FA
:101EE0005B0310922103109222031092230310929D
:101EF0002403E0915B03F0915C03EE0FFF1FEE0FF4
:101F0000FF1FEB5CFC4F6081718182819381D0C0A7
:101F1000C0905703D0905803E0905903F0905A03B3
:101F200020E030E0A901C701B6010E94052E2197EB
:101F3000882309F4A2C0FE01EE0FFF1FEE0FFF1F62
:101F4000EB5CFC4F80809180A280B380A50194015E
:101F5000C701B6010E94052E87FF31C0A50194017B
:101F600060E070E08CED93EC0E94092E20E030E000
:101F700040E451E40E94092E20E030E040E05FE3BD
:101F80000E94B42F9B01AC0160E070E080E090E41F
:101F90000E9417309B01AC01C501B4010E94B42F0F
:101FA0009B01AC01C701B6010E94052E87FF07C047
:101FB000A701960160E070E08CED93E439C0A501C3
:101FC0009401C701B6010E94B02F18160CF055C03D
:101FD000A501940160E070E08CED93E40E94092E6D
:101FE00020E030E040E451E40E94092E20E030E09F
:101FF00040E05FE30E94B42F9B01AC0160E070E021
:1020000080E090E40E9417309B01AC01C501B4014F
:102010000E94B42F9B01AC01C701B6010E94B02FF2
:1020200018165CF5A701960160E070E08CED93EC6A
:102030000E94092E20E030E040E451E40E94092E85
:1020400020E030E040E05FE30E94B42F9B01AC0150
:1020500060E070E080E090E40E9417309B01AC01EA
:10206000C701B6010E94B42F6093570370935803C1
:102070008093590390935A0313C0FE01EE0FFF1F84
:10208000EE0FFF1FEB5CFC4F80819181A281B38139
:102090008093570390935803A0935903B0935A0326
:1020A00060915703709158038091590390915A039E
:1020B00020910C0330910D032F3F4FEF340731F087
:1020C0002F5F3F4F30930D0320930C030E940C139E
:1020D0006B017C0120E034E244EF51E40E94052EC4
:1020E00087FF08C086EFC82E88E2D82E84EFE82E3E
:1020F00081E4F82E20E030E040E051E4C701B60171
:102100000E94B42F9B01AC0160E074E284E79BE481
:102110000E94092E6B017C010E94712E7093970022
:102120006093960020910A0230910B0240910C02BC
:1021300050910D02C701B6010E94B42F0E94712E6A
:10214000709399006093980080912003882309F48C
:1021500033C1C0901B03D0901C03E0901D03F0908E
:102160001E0320E030E0A901C701B6010E94B02F94
:102170001816D4F580910C0390910D038F3F2FEF2B
:10218000920729F0019690930D0380930C03C701E9
:10219000B6010E940C1320E030E040E051E40E94C0
:1021A000B42F9B01AC0160E074E284E79BE40E94E1
:1021B000092E6B017C010E94712E70939700609331
:1021C000960020910A0230910B0240910C0250912E
:1021D0000D02C701B6010E94B42F0E94712E7093A8
:1021E00099006093980008C0109297001092960092
:1021F0001092990010929800609115037091160347
:102200006F5F7F4F709316036093150320919600C4
:102210003091970080E090E0232BF1F0C091960080
:10222000D09197000E94A22E6B017C01BE0180E03C
:1022300090E00E94A22E9B01AC0160911703709167
:1022400018038091190390911A030E94092E20E02F
:102250003FEF4FE757E410C00E94A22E6B017C01B4
:1022600020E030EE4FEF54E46091170370911803B3
:102270008091190390911A030E94B42F9B01AC0125
:10228000C701B6010E94B02F87FD96C0809113034D
:102290008F5F8093130390E02091D8033091D9038E
:1022A00082179307A0F08091E303882319F010921E
:1022B00013030DC0809171008D7F80937100809118
:1022C00090008F7780939000109220037DC08091C2
:1022D0001403C0911303811128C0C090DD03D09076
:1022E000DE03E090DF03F090E00320E030E0A9019E
:1022F000C701B6010E94B02F1816BCF481E080938C
:10230000140310921B0310921C0310921D031092D1
:102310001E03C0921703D0921803E0921903F092A3
:102320001A03C150C093130343C0109214031092B8
:102330000D0310920C03E091DA03F091DB0348E007
:10234000C49FE00DF11D112480819181A281B38190
:1023500080931B0390931C03A0931D03B0931E0353
:1023600020E030E040E85EE36481758186819781FA
:102370000E94B42F6B017C0120E030E048EC52E475
:1023800060910E0270910F028091100290911102E3
:102390000E94092E9B01AC01C701B6010E94B42F17
:1023A00060931703709318038093190390931A0393
:1023B00010921603109215038091DC0380FD04C077
:1023C0001092200310921F03FF91EF91DF91CF91A4
:1023D000BF91AF919F918F917F916F915F914F913D
:1023E0003F912F91FF90EF90DF90CF90BF90AF90F3
:1023F0009F908F907F906F905F904F900F900FBE47
:102400000F901F901895CF92DF92EF92FF92CF938B
:10241000DF936B017C01EA0180910E03811102C000
:102420000E94FE0D8091DC0380FF46C080915D0319
:1024300090915E0308970CF03FC0809171008D7FF2
:10244000809371008091200381110E94180E81E019
:1024500080931F0310920D0310920C0320E030E0D4
:10246000A901C701B6010E94B02F1816DCF48091B3
:102470005D0390915E03FC01EE0FFF1FEE0FFF1F47
:10248000EB5CFC4FC082D182E282F382FC01EE0F52
:10249000FF1FEB5DFC4FD183C083019690935E03D9
:1024A00080935D03809171008260809371008091C0
:1024B0009000806880939000DF91CF91FF90EF9023
:1024C000DF90CF9008958F929F92AF92BF92CF925C
:1024D000DF92EF92FF920F931F93CF93DF93EC0164
:1024E0007B01D42E4801590180910E03811102C055
:1024F0000E94FE0D8091DC0380FF6BC08091710013
:102500008D7F8093710080911F0381110E94180EAE
:1025100081E080932003D093DB03C093DA03F09231
:10252000D903E092D803D092E3038092DD03909226
:10253000DE03A092DF03B092E00310922103109219
:102540002203109223031092240310921303888114
:102550009981AA81BB8180931B0390931C03A09354
:102560001D03B0931E0320E030E040E85EE36C8181
:102570007D818E819F810E94B42F6B017C0120E0C0
:1025800030E048EC52E460910E0270910F028091AD
:102590001002909111020E94092E9B01AC01C7010B
:1025A000B6010E94B42F60931703709318038093B1
:1025B000190390931A031092160310921503809139
:1025C0007100826080937100809190008068809398
:1025D0009000DF91CF911F910F91FF90EF90DF90CE
:1025E000CF90BF90AF909F908F90089580915F03A0
:1025F00090E0019666E070E00E94823180935F0374
:10260000089580915F0390E0019766E070E00E947A
:10261000823180935F0308958F929F92AF92BF9211
:10262000CF92DF92EF92FF920F931F93CF93DF939E
:102630006B017C01C0910C03D0910D03BE0180E0C1
:1026400090E00E94A22E4B015C01A701960160E080
:1026500070E08CE594E40E94092E9B01AC01C50159
:10266000B4010E94B42F0E94762E20915F03233084
:1026700009F473C028F4222351F02130E9F02CC171
:10268000243009F4A0C0253009F4E0C025C180E061
:1026900090E0A0E0BFE380930A0290930B02A09326
:1026A0000C02B0930D0210920F03109210031092BF
:1026B00011031092120310C110920F031092100315
:1026C00010921103109212036431710540F46A30C4
:1026D000710560F520E030E040E85EE32BC0693C26
:1026E000710508F0AAC080E090E00E94A22E20E0D0
:1026F00030E040EA51E40E94A02D20E030E044E3C5
:1027000053E40E94092E9B01AC010E94B42F20E0EB
:1027100030E040E05EE30E94B42F9B01AC0160E03A
:1027200070E080E09EE30E94A02D44C020E030E0F5
:1027300040E05FE3C701B6010E94B42F6B017C014A
:1027400080E090E0A0E0BEE380930A0290930B0249
:10275000A0930C02B0930D02BFC010920F03109211
:10276000100310921103109212034AE0469F900149
:10277000479F300D1124C90168EB7BE00E946E3148
:10278000BC016C5D754077FF03C07195619571095F
:10279000882777FD8095982F0E94A42E2EE333EC96
:1027A0004EE259E30E94B42F20E030E040EC5EE3BB
:1027B0000E94A12D60930A0270930B0280930C0279
:1027C00090930D0289C010920F0310921003109283
:1027D000110310921203CE0183709927892BE1F027
:1027E000BE016170772780E090E00E94A22E20E079
:1027F00030E040E05EE30E94B42F20E030E040E4AF
:102800005FE30E94A12D60930A0270930B028093F4
:102810000C0290930D020CC080E090E0A0E0BFE3BA
:1028200080930A0290930B02A0930C02B0930D02C6
:10283000C770DD27CD2B09F04FC010920A0210920D
:102840000B0210920C0210920D0246C010920F0360
:1028500010921003109211031092120300E010E086
:1028600020E03FE300930A0210930B0220930C0236
:1028700030930D026739710578F180E090E00E9495
:10288000A22E20E030E047E153E40E94A02D20E09A
:1028900030E04AE754E40E94092E20E030E048E4AA
:1028A00052E40E94B42F20E030E040EA51E40E945C
:1028B000E62E0E94712E660F771F660F771FFB01B1
:1028C000E357FD4F2081318142815381C701B60119
:1028D0000E94B42F6B017C01C701B601DF91CF913B
:1028E0001F910F91FF90EF90DF90CF90BF90AF902E
:1028F0009F908F900895809168030895CF93DF9300
:1029000000D01F92CDB7DEB79C018091E8038430E0
:1029100019F593E099833B832A839093E9008FEF25
:102920009091E800815095FD06C095ED9A95F1F7DC
:1029300000008111F5CF8091E80085FF0DC040E0D7
:1029400050E063E070E0CE0101960E94B7168091DE
:10295000E8008E778093E8000F900F900F90DF9142
:10296000CF910895CF93DF9300D01F92CDB7DEB7FC
:102970002091E803243021F522E029839B838A8378
:1029800083E08093E9008FEF9091E800815095FDFE
:1029900006C095ED9A95F1F700008111F5CF809171
:1029A000E80085FF0DC040E050E063E070E0CE013C
:1029B00001960E94B7168091E8008E778093E80018
:1029C0000F900F900F90DF91CF9108952091E80321
:1029D0002430F1F422E02093E9002FEF3091E80059
:1029E000215035FD06C035ED3A95F1F70000211173
:1029F000F5CF2091E80025FF0BC040E050E065E0F6
:102A000070E00E94B7168091E8008E778093E8000E
:102A10000895CF93DF932091E803243039F521E026
:102A20002093E9002FEF3091E800215035FD06C0DA
:102A300035ED3A95F1F700002111F5CF2091E8002E
:102A400025FF14C0EC0140E050E068E070E00E9417
:102A5000B7168091E8008E778093E80088E0FE0149
:102A6000A0E6B3E001900D928A95E1F7DF91CF9156
:102A700008958091E703811109C00E944C180E94BB
:102A8000A9188091E20084608093E200089510927A
:102A9000E7030895089508950C94A72742E061EC98
:102AA00081E00E94C61742E061EC82E00E94C617F6
:102AB00042E061EC83E00C94C6178091EA03833016
:102AC00009F453C030F4813071F0823009F48CC0C5
:102AD00008958A3009F478C08B3009F45EC08930DB
:102AE00009F09AC020C08091E903813A09F094C0AE
:102AF0008091E800877F8093E8008091ED039091BA
:102B0000EE03892B21F468E080E693E003C060E0E7
:102B100080E090E070E00E9402178091E8008B77DF
:102B20008093E80008958091E903813209F074C030
:102B30008091ED039091EE03892B09F06DC0809197
:102B4000E800877F8093E8008091E80082FD05C05F
:102B50008091E8038111F8CF5FC08091F1008093EC
:102B600068038091E8008B7753C08091E903813A34
:102B700009F052C08091ED039091EE03892B09F08A
:102B80004BC08091E800877F8093E8008091E80047
:102B900080FFFCCF80911C0236C08091E903813216
:102BA000D9F58091ED039091EE03892BA9F58091E1
:102BB000E800877F8093E8000E94FB178091EB0379
:102BC00080931C020C946C218091E903813221F5E1
:102BD0008091E800877F8093E8000E94FB17809136
:102BE000EC038093690308958091E903813AA1F48D
:102BF0008091E800877F8093E8008091E80080FF63
:102C0000FCCF809169038093F1008091E8008E777A
:102C10008093E8000C94FB17089584B7877F84BFE6
:102C200088E10FB6F89480936000109260000FBEA8
:102C300090E080E80FB6F894809361009093610073
:102C40000FBE0E949E1B0E944C180E94A9188091E2
:102C5000E20084608093E20078940E942F1B0E941F
:102C6000A01B82E192E00E944A1B8091E80385301C
:102C700069F40E9461278091E6038823B1F30E94E2
:102C80008F27882391F30E94A116EFCF0E94A81BE3
:102C9000ECCF292F332723303105C9F064F42130DC
:102CA000310581F02230310509F043C084E590E020
:102CB00020ED39E042C021323105F1F022323105F8
:102CC00041F137C082E190E024E23AE036C0992732
:102CD0008130910541F08230910541F0892B49F511
:102CE000ECECF9E005C0EEE9F9E002C0E2E7F9E05A
:102CF000849190E09F0121C06330D8F4E62FF0E08A
:102D0000EE0FFF1FEA51FD4F2081318189E090E0F5
:102D100014C0633070F470E0FB01EE0FFF1FE0524F
:102D2000FD4F20813181FB01E352FD4F808190E016
:102D300004C080E090E020E030E0FA01318320839D
:102D4000089580E189BD82E189BD09B400FEFDCF0F
:102D50008091D8008F7D8093D8008091E0008260C0
:102D60008093E0008091E00081FDFCCF0895CF9238
:102D7000DF92EF92FF920F931F93CF93DF93EC01BB
:102D80008B016A010E941A18811133C0C114D10449
:102D900039F0F60180819181081B190BC80FD91FEA
:102DA000E12CF12C0115110519F18091E80085FD48
:102DB00016C08091E8008E778093E800C114D1049A
:102DC00049F0F60180819181E80EF91EF182E082DE
:102DD00085E00FC00E941A18882321F30AC0899148
:102DE0008093F10001501109FFEFEF1AFF0ADACFCB
:102DF00080E0DF91CF911F910F91FF90EF90DF90D6
:102E0000CF9008952091EF033091F00326173707F4
:102E100048F06115710539F42091E8002E77209370
:102E2000E80001C0B90140E061157105A9F12091E8
:102E3000E803222309F443C0253009F442C020915D
:102E4000E80023FD40C02091E80022FD32C020911F
:102E5000E80020FFE9CF4091F3002091F20030E03C
:102E6000342BFC01CF016115710559F02830310573
:102E700040F481918093F100615071092F5F3F4FC1
:102E8000F1CF41E02830310509F040E02091E80021
:102E90002E772093E800C8CF4111C9CF0AC0809196
:102EA000E803882361F0853061F08091E80083FDBC
:102EB0000AC08091E80082FFF2CF80E0089582E0AE
:102EC000089583E0089581E008952091EF03309103
:102ED000F0032617370748F06115710539F4209182
:102EE000E8002E772093E80001C0B901FC0120E042
:102EF0006115710591F18091E803882309F440C0C0
:102F0000853009F43FC08091E80083FD3DC0809189
:102F1000E80082FD2FC08091E80080FFE9CF20917A
:102F2000F3008091F20090E0922B6115710559F049
:102F30008830910540F424912093F100319661503E
:102F400071090196F2CF21E0089709F020E0809105
:102F5000E8008E778093E800CBCF2111CCCF0AC058
:102F60008091E803882361F0853061F08091E8006A
:102F700083FD0AC08091E80082FFF2CF80E00895CF
:102F800082E0089583E0089581E00895982F9730B6
:102F900058F59093E900981739F07091EC00209162
:102FA000ED005091F00003C0242F762F50E021FF58
:102FB00019C03091EB003E7F3093EB003091ED0073
:102FC0003D7F3093ED003091EB0031603093EB00AA
:102FD0007093EC002093ED005093F0002091EE00F0
:102FE00027FF07C09F5FD3CF8F708093E90081E0F8
:102FF000089580E008958091E90387FF11C08091D2
:10300000E80082FD05C08091E8038111F8CF11C06E
:103010008091E8008B770BC08091E803882349F00A
:103020008091E80080FFF8CF8091E8008E77809350
:10303000E80008952091E4003091E50095E6409184
:10304000EC00842F817040FF22C08091E80080FD59
:103050001CC08091E803882391F0853091F0809125
:10306000EB0085FD10C04091E4005091E50042174F
:10307000530729F39A01915011F784E0089582E0F3
:10308000089583E0089581E0089580E008954091D7
:10309000E80042FFDECF08950E94BA180E94C218CD
:1030A000E0EEF0E0808181608083E8EDF0E08081F7
:1030B0008F77808319BCA7EDB0E08C918E7F8C93C5
:1030C00080818F7E80831092E70308950F931F9372
:1030D000CF93DF930E94BA180E94C218C8EDD0E0C7
:1030E00088818F77888388818068888388818F7DB5
:1030F000888319BC1092E8031092E4031092E6034F
:103100001092E50300EE10E0F80180818B7F808350
:1031100088818160888342E060E080E00E94C61779
:10312000E1EEF0E080818E7F8083E2EEF0E080814E
:1031300081608083808188608083F80180818E7FB8
:103140008083888180618883DF91CF911F910F9167
:103150000895E8EDF0E080818F7E8083E7EDF0E078
:1031600080818160808384E082BF81E08093E70377
:103170000C946618E8EDF0E080818E7F80831092D9
:10318000E20008951092DA001092E10008951F9273
:103190000F920FB60F9211242F933F934F935F938B
:1031A0006F937F938F939F93AF93BF93EF93FF930F
:1031B0008091E10082FF0BC08091E20082FF07C096
:1031C0008091E1008B7F8093E1000E942E1B809113
:1031D000DA0080FF1FC08091D80080FF1BC0809163
:1031E000DA008E7F8093DA008091D90080FF0DC0D5
:1031F00080E189BD82E189BD09B400FEFDCF81E097
:103200008093E8030E94391505C019BC1092E803A9
:103210000E9447158091E10080FF19C08091E20073
:1032200080FF15C08091E2008E7F8093E200809144
:10323000E20080618093E2008091D80080628093F8
:10324000D80019BC85E08093E8030E944B1580915B
:10325000E10084FF30C08091E20084FF2CC080E157
:1032600089BD82E189BD09B400FEFDCF8091D800FF
:103270008F7D8093D8008091E1008F7E8093E10064
:103280008091E2008F7E8093E2008091E200816075
:103290008093E2008091E403882311F084E007C06A
:1032A0008091E30087FD02C081E001C083E080934C
:1032B000E8030E944C158091E10083FF29C08091B2
:1032C000E20083FF25C08091E100877F8093E100C9
:1032D00082E08093E8031092E4038091E1008E7F06
:1032E0008093E1008091E2008E7F8093E2008091E4
:1032F000E20080618093E20042E060E080E00E94B2
:10330000C6178091F00088608093F0000E944A15F3
:10331000FF91EF91BF91AF919F918F917F916F91AD
:103320005F914F913F912F910F900FBE0F901F9083
:1033300018951F920F920FB60F9211242F933F935F
:103340004F935F936F937F938F939F93AF93BF93AD
:10335000CF93DF93EF93FF93C091E900CF708091FB
:10336000EC00D82FD17080FDD0E81092E900809158
:10337000F000877F8093F00078940E94DD1910920E
:10338000E9008091F00088608093F000CD2BCF7031
:10339000C093E900FF91EF91DF91CF91BF91AF9181
:1033A0009F918F917F916F915F914F913F912F915D
:1033B0000F900FBE0F901F9018951F93CF93DF9320
:1033C000CDB7DEB7AA970FB6F894DEBF0FBECDBF5C
:1033D000E9EEF3E088E08E0F9091F10091938E1367
:1033E000FBCF0E945D158091E80083FF1FC1809193
:1033F000E9039091EA03492F50E04A30510508F063
:1034000015C1FA01EE59FF4F0C949631803881F0C6
:10341000823809F00BC18091ED038F708093E90031
:103420008091EB0085FB882780F91092E90006C0A7
:103430008091E5039091E603911182609091E800FC
:10344000977F9093E8008093F1001092F100C8C03C
:10345000282F2D7F09F0EAC0882319F0823061F00F
:10346000E5C08091EB03813009F0E0C0933009F0B2
:1034700080E08093E6032BC08091EB03811127C08D
:103480008091ED038F7009F4D1C08093E900209101
:10349000EB0020FF1CC0933021F48091EB00806290
:1034A00014C09091EB0090619093EB0021E030E02C
:1034B000A90102C0440F551F8A95E2F74093EA0024
:1034C0001092EA008091EB0088608093EB001092EC
:1034D000E9008091E800877F86C08111A7C0109124
:1034E000EB031F778091E3008078812B8093E300CA
:1034F0008091E800877F8093E8000E94FB1780910D
:10350000E80080FFFCCF8091E30080688093E300B7
:10351000111102C082E001C083E08093E80386C0FD
:103520008058823008F082C08091EB039091EC03C8
:103530008C3D53E0950779F583E08A838AE289839D
:103540004FB7F894DE01139620E03EE051E2E32FFE
:10355000F0E050935700E49120FF03C0E295EF7034
:103560003F5FEF708E2F90E0EA3010F0C79601C0F9
:10357000C0968D939D932F5F243149F74FBF809163
:10358000E800877F8093E8006AE270E0CE01019650
:103590000E94021714C0AE014F5F5F4F6091ED03B0
:1035A0000E944916BC01009709F440C09091E800C0
:1035B000977F9093E80089819A810E946517809196
:1035C000E8008B778093E80031C0803879F58091EE
:1035D000E800877F8093E8008091E4038093F10006
:1035E0008091E8008E778093E8000E94FB171EC050
:1035F00081111CC09091EB039230C0F48091E800DF
:10360000877F8093E8009093E4030E94FB178091EA
:10361000E403811106C08091E30087FD02C081E0D0
:1036200001C084E08093E8030E944E158091E80079
:1036300083FF0AC08091E800877F8093E800809133
:10364000EB0080628093EB00AA960FB6F894DEBF81
:103650000FBECDBFDF91CF911F9108950895CF93F5
:103660008091E8038823A1F0C091E900CF70909188
:10367000EC00892F817090FD80E8C82B1092E90042
:103680008091E80083FD0E94DD19CF70C093E900AE
:10369000CF91089590936F0380936E030895E09106
:1036A0006E03F0916F03309721F00190F081E02DCF
:1036B000099480E00895E0916E03F0916F033097D4
:1036C00021F00280F381E02D09940895E0916E03CA
:1036D000F0916F03309721F00480F581E02D09947B
:1036E000089520916C0330916D038217930771F058
:1036F00090936D0380936C03E0916E03F0916F03E0
:10370000309721F00680F781E02D099408952091EB
:103710006A0330916B038217930771F090936B03E8
:1037200080936A03E0916E03F0916F03309721F06C
:103730000084F185E02D0994089508950C949D1B53
:103740000E94DB270E94D20B0E9461280C94092D55
:103750004F925F927F928F929F92AF92BF92CF9241
:10376000DF92EF92FF920F931F93CF93DF93CDB72A
:10377000DEB72A970FB6F894DEBF0FBECDBF0E940A
:10378000AD0C91E7C92E93E0D92E00E010E0AA24F9
:10379000A394B12C702E802F0E94E60D4C01F601EF
:1037A000419051906F014826592641145104B1F4BB
:1037B0000F5F1F4F0530110569F78FEF89838A83EB
:1037C0001B820E94E4278160782F9D838C8349812E
:1037D0005A816B818D810E94611C3AC08091C70320
:1037E00081FD0E94EF0D20E030E07501022E02C045
:1037F000EE0CFF1C0A94E2F7C70184219521892B66
:1038000009F12E837F828E209F2091E0892809F480
:1038100090E098870E94E4278160782F9A878987B3
:103820004E815F8168858A850E94611C000F111F8F
:10383000F801EF58FC4F80819181E826F926F1824A
:10384000E08206C02F5F3F4F2C30310571F6B0CFBC
:103850000E94482A109170030E944F1B1817D9F03C
:103860000E944F1B809370032A960FB6F894DEBF18
:103870000FBECDBFDF91CF911F910F91FF90EF90C1
:10388000DF90CF90BF90AF909F908F907F905F9090
:103890004F900C940A0B2A960FB6F894DEBF0FBE19
:1038A000CDBFDF91CF911F910F91FF90EF90DF90EF
:1038B000CF90BF90AF909F908F907F905F904F90F0
:1038C0000895CF93DF93CDB7DEB72B970FB6F8945B
:1038D000DEBF0FBECDBF4F83588769877A878B873E
:1038E000DE01119686E0FD0111928A95E9F785E0E7
:1038F000FE01379601900D928A95E1F749815A8130
:103900006B817C818D819E810E9406242B960FB64F
:10391000F894DEBF0FBECDBFDF91CF910895CF9356
:10392000882309F4C2C0C82F823859F40E944F1B63
:1039300081FDBBC089E30E94AF260E94322789E344
:103940000CC0833879F40E944F1B80FDAEC083E524
:103950000E94AF260E94322783E50E94CC26CF9199
:103960000C943227843859F40E944F1B82FD9DC06D
:1039700087E40E94AF260E94322787E4EECF8CEFC7
:103980008C0F813A48F48C2F0E94712C81118DC0CC
:103990008C2F0E94AF26E3CF80E28C0F883048F452
:1039A000C77081E001C0880FCA95EAF70E94EB2634
:1039B000D6CF8BE58C0F833078F4C53A29F0C63A20
:1039C00031F083E890E005C081E890E002C082E831
:1039D00090E0CF910C94711B88E58C0F833108F037
:1039E00064C0C83A39F1C93A41F1CA3A49F1CB3A0F
:1039F00051F1CC3A59F1CD3A61F1C03B69F1CE3A7F
:103A000071F1CF3A79F1C13B81F1C23B89F1C33BFE
:103A100091F1C43B99F1C53BA1F1C63BA9F1C73B6C
:103A2000B1F1C83BB9F1C93BC1F1CA3BC9F180E072
:103A300090E038C082EE90E035C089EE90E032C070
:103A40008AEE90E02FC085EB90E02CC086EB90E0F2
:103A500029C087EB90E026C08CEC90E023C08DEC71
:103A600090E020C083E891E01DC08AE891E01AC090
:103A700082E991E017C084E991E014C081E292E00C
:103A800011C083E292E00EC084E292E00BC085E2B6
:103A900092E008C086E292E005C087E292E002C0B0
:103AA0008AE292E0CF910C94871BCF9108958823EE
:103AB00009F44BC0823859F40E944F1B81FF45C066
:103AC00089E30E94AF260E94322789E30CC0833825
:103AD00071F40E944F1B80FF38C083E50E94AF261F
:103AE0000E94322783E50E94CC260C94322784382A
:103AF00059F40E944F1B82FF28C087E40E94AF2622
:103B00000E94322787E4EFCF9CEF980F913A58F349
:103B100090E2980F983050F4877091E001C0990FAF
:103B20008A95EAF7892F0E94F126DFCF9BE5980F4F
:103B3000933020F480E090E00C94711B885A83311C
:103B400020F480E090E00C94871B0895882321F0F6
:103B50000E94EB260C9432270895882321F00E94BE
:103B6000F1260C9432270895BF92CF92DF92EF9204
:103B7000FF920F931F93CF93DF9300D000D000D01C
:103B8000CDB7DEB725E0FC01DE01119601900D9264
:103B90002A95E1F7FC01D0801181028125812295CF
:103BA0002F7043815481452B09F472C31F3F21F4C8
:103BB000FFEFDF1609F46CC37C012E830E94D3074C
:103BC000D9821A8369817A81802F0E94AB26182FAF
:103BD000B92E0E9460260E9427252E81002319F00D
:103BE0000E9408272E81EB2DE295EF70F0E0E4595A
:103BF000FF4F0C9496318B2D807F9B2D9F70F92E5B
:103C0000882319F0F29480EFF822002389F0FF2036
:103C100009F47CC280E2810F883020F48F2D0E944D
:103C2000EB2603C08F2D0E94FB260E9432276EC216
:103C3000812F0E94571DFF2009F42AC3105E8F2D8B
:103C4000183018F40E94F12602C00E94012726961F
:103C50000FB6F894DEBF0FBECDBFDF91CF911F919D
:103C60000F91FF90EF90DF90CF90BF900C94322790
:103C70008B2D807F9B2D9F70803211F4892F03C084
:103C8000892F8295807F112319F0113011F12BC0FB
:103C90000023A9F0222389F1213079F526960FB669
:103CA000F894DEBF0FBECDBFDF91CF911F910F9172
:103CB000FF90EF90DF90CF90BF900C941B272223B2
:103CC00019F0213009F4E4C28E830E941E278E81F0
:103CD0009BC1002321F0263008F0DAC20EC0253047
:103CE00008F0D6C291C10023C9F0222331F0F701B8
:103CF000958190FF0BC29F70958326960FB6F8941E
:103D0000DEBF0FBECDBFDF91CF911F910F91FF900E
:103D1000EF90DF90CF90BF900C94A61D222309F462
:103D200073C109C22B2D26952695237030E02115ED
:103D3000310521F021303105D1F0AAC2002321F054
:103D4000812F9B2D937002C080E090E026960FB6E5
:103D5000F894DEBF0FBECDBFDF91CF911F910F91C1
:103D6000FF90EF90DF90CF90BF900C94711B0023D9
:103D700021F0812F9B2D937002C080E090E0269669
:103D80000FB6F894DEBF0FBECDBFDF91CF911F916C
:103D90000F91FF90EF90DF90CF90BF900C94871B16
:103DA000812F002319F00E94502902C00E94B829D7
:103DB00026960FB6F894DEBF0FBECDBFDF91CF9130
:103DC0001F910F91FF90EF90DF90CF90BF900C94D8
:103DD0003D2A8B2D837009F07BC0011159C2812FC0
:103DE000829586958770880F880F912F9F70C92EB6
:103DF000D12CE12CF12C082E04C0CC0CDD1CEE1CC7
:103E0000FF1C0A94D2F714FF12C04FE050E060E0AC
:103E100070E004C0440F551F661F771F8A95D2F7C4
:103E2000CB01BA01609570958095909503C060E0D4
:103E300070E0CB012B2D269526952370422F50E064
:103E400042305105D9F04330510569F16C297D2983
:103E50008E299F294130510551F126960FB6F894CD
:103E6000DEBF0FBECDBFDF91CF911F910F91FF90AD
:103E7000EF90DF90CF90BF900C944E256C297D2958
:103E80008E299F2926960FB6F894DEBF0FBECDBFB0
:103E9000DF91CF911F910F91FF90EF90DF90CF9026
:103EA000BF900C946A250E944E25C701B601269644
:103EB0000FB6F894DEBF0FBECDBFDF91CF911F913B
:103EC0000F91FF90EF90DF90CF90BF900C94322530
:103ED000002319F08B2D817001C08695882309F489
:103EE000D7C1812F829586958770880F880F912F73
:103EF0009F70C92ED12CE12CF12C082E04C0CC0CC3
:103F0000DD1CEE1CFF1C0A94D2F714FF12C04FE018
:103F100050E060E070E004C0440F551F661F771F3B
:103F20008A95D2F7CB01BA016095709580959095EE
:103F300003C060E070E0CB012B2D26952695237001
:103F4000422F50E042305105D9F04330510569F11C
:103F50006C297D298E299F294130510551F12696E2
:103F60000FB6F894DEBF0FBECDBFDF91CF911F918A
:103F70000F91FF90EF90DF90CF90BF900C94282688
:103F80006C297D298E299F2926960FB6F894DEBFCD
:103F90000FBECDBFDF91CF911F910F91FF90EF909A
:103FA000DF90CF90BF900C9444260E942826C70132
:103FB000B60126960FB6F894DEBF0FBECDBFDF91D7
:103FC000CF911F910F91FF90EF90DF90CF90BF9016
:103FD0000C940C26103F49F118F4103E48F491C09F
:103FE000123F09F453C0E8F1133F09F464C089C0DB
:103FF0001F708B2D8F71002321F00E94A525812F2A
:104000007CCE0E94C625812F26960FB6F894DEBF7F
:104010000FBECDBFDF91CF911F910F91FF90EF9019
:10402000DF90CF90BF900C94AD1D0023B1F02530F0
:1040300008F02EC18B2D8F7126960FB6F894DEBF37
:104040000FBECDBFDF91CF911F910F91FF90EF90E9
:10405000DF90CF90BF900C94EB25263008F018C16C
:10406000E9CF0023A9F08B2D8F7126960FB6F89417
:10407000DEBF0FBECDBFDF91CF911F910F91FF909B
:10408000EF90DF90CF90BF900C94A525002359F3BB
:104090008B2D8F7126960FB6F894DEBF0FBECDBF65
:1040A000DF91CF911F910F91FF90EF90DF90CF9014
:1040B000BF900C94C625002399F08B2D8F71269606
:1040C0000FB6F894DEBF0FBECDBFDF91CF911F9129
:1040D0000F91FF90EF90DF90CF90BF900C949025C0
:1040E00026960FB6F894DEBF0FBECDBFDF91CF91FD
:1040F0001F910F91FF90EF90DF90CF90BF900C94A5
:1041000086250023A9F0222309F4ADCF812F26961E
:104110000FB6F894DEBF0FBECDBFDF91CF911F91D8
:104120000F91FF90EF90DF90CF90BF900C948F1C79
:10413000222309F4ADCF812F26960FB6F894DEBF67
:104140000FBECDBFDF91CF911F910F91FF90EF90E8
:10415000DF90CF90BF900C94571D4B2D4F70612F67
:10416000C7010E940B0626960FB6F894DEBF0FBE5D
:10417000CDBFDF91CF911F910F91FF90EF90DF9016
:10418000CF90BF900C94AA24011182C09B2D9F70E8
:10419000492F50E04230510509F443C0C4F44115A1
:1041A000510571F14130510509F072C026960FB6E4
:1041B000F894DEBF0FBECDBFDF91CF911F910F915D
:1041C000FF90EF90DF90CF90BF900C94312D433053
:1041D0005105C1F14430510509F05AC0812F26968E
:1041E0000FB6F894DEBF0FBECDBFDF91CF911F9108
:1041F0000F91FF90EF90DF90CF90BF900C94832DA4
:1042000026960FB6F894DEBF0FBECDBFDF91CF91DB
:104210001F910F91FF90EF90DF90CF90BF900C9483
:104220001A2D26960FB6F894DEBF0FBECDBFDF91D4
:10423000CF911F910F91FF90EF90DF90CF90BF90A3
:104240000C944D2D26960FB6F894DEBF0FBECDBF51
:10425000DF91CF911F910F91FF90EF90DF90CF9062
:10426000BF900C94602D4B2D4F70612FC701269687
:104270000FB6F894DEBF0FBECDBFDF91CF911F9177
:104280000F91FF90EF90DF90CF90BF900C94D507E7
:1042900026960FB6F894DEBF0FBECDBFDF91CF914B
:1042A0001F910F91FF90EF90DF90CF90BF900895F6
:1042B0000E9408270E9418270E94DD260E943227AC
:1042C0000E94EE2A0E943D2A80E090E00E94711B2D
:1042D00080E090E00C94871B0E94F8260C945821F3
:1042E0000E94A026292F22952F7030E02C30310516
:1042F0004CF42A3031056CF422503109223031055A
:1043000088F407C02C30310549F02F30310531F0E9
:1043100009C0803E48F0803F29F406C093FB8827FF
:1043200080F9089580E0089581E00895CF93DF93A8
:1043300000D000D01F92CDB7DEB70F900F900F9036
:104340000F900F90DF91CF910895CF93DF9300D01E
:1043500000D000D0CDB7DEB726960FB6F894DEBFFA
:104360000FBECDBFDF91CF9108951F93CF93DF9301
:10437000C0917B0316E080917C03C81799F0D0E0D0
:104380001C9FF0011D9FF00D1124E358FC4F40814C
:10439000518162817381848195810E94A52121963A
:1043A000C770E9CFDF91CF911F9108954091AD0380
:1043B0005091AE036091AF037091B0038091B1034F
:1043C0009091B2030C94A5218091B20382958F70D5
:1043D00009F054C08091AF03882309F44FC0809145
:1043E0007B03A0917C036091AD037091AE0340917B
:1043F000B0035091B103B6E08A1709F43FC090E0D2
:1044000041155105C1F17F3F11F46F3FA1F1B89FF4
:10441000F001B99FF00D1124E358FC4F2181721374
:104420002AC02081621327C02281211124C0238148
:1044300034812417350710F421503109241B350B22
:10444000283C3105C0F42091B2032F7020612093E5
:10445000B20326E0289FF001299FF00D1124EE57AA
:10446000FC4F80818F70806180838DEA93E00E9491
:10447000B41D0C94B52101968770BECF0895CF92DC
:10448000DF92EF92FF920F931F93CF93DF93CDB7FD
:10449000DEB762970FB6F894DEBF0FBECDBF8C01BA
:1044A00085E0F801DE011D9601900D928A95E1F7F5
:1044B000D8014C9111965C91119712966C911297BC
:1044C0001396CD90DC9014973091AD037091AE03AC
:1044D0008091B0039091B103009709F46BC17F3FC5
:1044E00019F43F3F09F466C1E090AF03EE2009F4F0
:1044F000C0C02091B203C816D90628F0F601E81B07
:10450000F90BCF0104C0809590958C0D9D1DFF2463
:10451000F394883C910578F0F12C207F09F0C6C017
:104520007C2DD98AC88A89890E9496218DEA93E0D8
:104530000E94B41DB1C0822F807F09F046C0751360
:1045400014C0341312C0611110C02F702061209369
:10455000B2030E94D6218DEA93E00E94B41D80919F
:10456000B203D80115968C932EC0CD2819F15F3F68
:1045700011F44F3FF9F0F62E61111CC080917B03BE
:1045800020917C0336E0821709F45AC090E0389FEE
:10459000F001399FF00D1124E358FC4F718157133E
:1045A00006C07081471303C07281711103C0019668
:1045B0008770E9CFF62E662309F418C18091B20303
:1045C00081608093B203F12C11C1751308C03413BC
:1045D00006C0611104C08091B203D801C3C04D87E9
:1045E0005E878D859E856A8B0E9470216A898823EB
:1045F000E1F16623D1F12091B203822F82958F7071
:1046000090E0029774F08091AD039091AE0398878B
:104610008F831986DB86CA862C87CE0107960E9477
:10462000B41D86E0F801ADEAB3E001900D928A95E1
:10463000E1F70E94E4210E94D621FF24F394D6C022
:104640004D875E878D859E850E94A026292F229505
:104650002F7030E0223031050CF0BCC09F7009F0A3
:10466000B6C0805E883008F4C1C0C8010E94B41D85
:10467000E4CFC816D90608F453C0F601E81BF90BBD
:10468000CF01883C910508F450C0F12C7C2DD98ACB
:10469000C88A89890E949621EDEAF3E086E0DF016D
:1046A0001D928A95E9F70E94D621A0C0751314C007
:1046B000341312C0611110C08091B203F8018583D8
:1046C000C8010E94B41D86E0EDEAF3E0DF011D920F
:1046D0008A95E9F7FE2C8AC04D875E878D859E8579
:1046E0006A8B0E9470216A89882309F4BECF6623F1
:1046F00009F4BBCF2091B203822F82958F7090E096
:1047000002970CF48ECF8091AD039091AE039A8303
:1047100089831B82DD82CC822E83CE0101967FCFDE
:10472000809590958C0D9D1DACCFF62E662309F4D7
:104730009CCF75132EC034132CC02091B20320FDE2
:104740001FC0822F82958F70D9F0D80115962C93B7
:1047500015978F3049F08F5F982F9295907F822F19
:104760008F70892B15968C93C8010E94B41D86E02A
:10477000F801ADEAB3E001900D928A95E1F793CF8D
:1047800086E0F801ADEAB3E001900D928A95E1F779
:104790002DC04D875E878D859E850E947021811179
:1047A00040CF8091B20381608093B203C8010E9420
:1047B000B41D1CC0662309F458CF4D875E878D85D4
:1047C0009E850E947021882309F44FCF2ACF811142
:1047D00048CF0CC0243031050CF047CF9F7009F44E
:1047E00040CFF8019581907F09F03BCF8F2D6296E5
:1047F0000FB6F894DEBF0FBECDBFDF91CF911F91F2
:104800000F91FF90EF90DF90CF9008951F93CF937B
:10481000DF93CDB7DEB72C970FB6F894DEBF0FBE8F
:10482000CDBF4F83588769877A878B879C87CE0156
:1048300007960E943F22882369F08F8198852A85F8
:104840003B85232BF1F19F3F09F063C08F3F09F0B7
:1048500060C037C086E0FE013796DE0111960190F8
:104860000D928A95E1F76F817885EA85FB8530970F
:1048700041F17F3F11F46F3F21F120917C0330E043
:10488000C90101968770992740917B0350E08417F6
:10489000950709F447C069837A83FD83EC8396E02A
:1048A000929FD001939FB00D1124A358BC4FFE01DD
:1048B000319601900D929A95E1F780937C030E94C6
:1048C000B52116E080917B0390917C038917C1F19B
:1048D000189FC001112483589C4F0E943F228823B7
:1048E00079F1E0917B031E9FF0011124E358FC4F06
:1048F0004081518162817381848195810E94A521CB
:1049000080917B0390E001968770992780937B03C9
:10491000D9CF4F81588569857A858B859C850E9482
:10492000A521CFCF0E946C2110927C0310927B03B3
:10493000EDEAF3E086E0DF011D928A95E9F7C1CF49
:104940002C960FB6F894DEBF0FBECDBFDF91CF918E
:104950001F910895EF92FF920F931F93CF93DF93D0
:104960008C01009709F46CC0F12CEE24E394E8016B
:104970002196F8018491843740F4843008F051C0C6
:10498000813081F0823019F15BC0853709F444C071
:10499000A8F19CE7980F903708F052C08F770E94DB
:1049A000571D41C00E5F1F4FFE01C49180E28C0F66
:1049B000883048F4C7708E2D01C0880FCA95EAF779
:1049C0000E940B2714C08C2F0E948F1C2DC00E5FDD
:1049D0001F4FFE01C49180E28C0F883058F4C770DD
:1049E0008E2D01C0880FCA95EAF70E9411270E94F8
:1049F00032271AC08C2F0E94571D16C00E5F1F4F02
:104A0000FE01C491CC2381F08FE99FE00197F1F77B
:104A100000C00000C150F6CF0E5F1F4FFE01F490A2
:104A200003C00E948F1C8E018F2D882309F49FCF15
:104A3000EFE9FFE03197F1F700C000008150F5CFBA
:104A4000DF91CF911F910F91FF90EF9008950895FE
:104A50006093B7037093B8038093B9039093BA033C
:104A60000C9458210F931F930091B7031091B80332
:104A70002091B9033091BA03DC01CB01802B912B3B
:104A8000A22BB32B8093B7039093B803A093B903E1
:104A9000B093BA031F910F910C9458210F931F9359
:104AA0000091B7031091B8032091B9033091BA0374
:104AB000DC01CB0180239123A223B3238093B7038E
:104AC0009093B803A093B903B093BA031F910F91C9
:104AD0000C9458210F931F930091B7031091B803C2
:104AE0002091B9033091BA03DC01CB0180279127D3
:104AF000A227B3278093B7039093B803A093B90379
:104B0000B093BA031F910F910C9458211092B303E4
:104B10001092B4031092B5031092B6030C9458216E
:104B200041E050E060E070E004C0440F551F661F94
:104B3000771F8A95D2F74093B3035093B4036093E1
:104B4000B5037093B6030C94582141E050E060E047
:104B500070E004C0440F551F661F771F8A95D2F777
:104B60008091B3039091B403A091B503B091B603C3
:104B7000482B592B6A2B7B2B4093B3035093B403E0
:104B80006093B5037093B6030C94582141E050E054
:104B900060E070E004C0440F551F661F771F8A95C0
:104BA000D2F740955095609570958091B3039091A0
:104BB000B403A091B503B091B603482359236A23E7
:104BC0007B234093B3035093B4036093B503709376
:104BD000B6030C94582141E050E060E070E004C05E
:104BE000440F551F661F771F8A95D2F78091B30334
:104BF0009091B403A091B503B091B603482759270B
:104C00006A277B274093B3035093B4036093B503A3
:104C10007093B6030C9458210F931F930091B30324
:104C20001091B4032091B5033091B603DC01CB01A0
:104C3000802B912BA22BB32B8093B3039093B403BF
:104C4000A093B503B093B6031F910F910C94582114
:104C50000F931F930091B3031091B4032091B503F8
:104C60003091B603DC01CB0180239123A223B3232F
:104C70008093B3039093B403A093B503B093B603AA
:104C80001F910F910C9458210F931F930091B30320
:104C90001091B4032091B5033091B603DC01CB0130
:104CA00080279127A227B3278093B3039093B4035F
:104CB000A093B503B093B6031F910F910C945821A4
:104CC0000895CF92DF92EF92FF920F931F93CF93AD
:104CD000DF938C01C090B703D090B803E090B90384
:104CE000F090BA038091B3039091B403A091B503FF
:104CF000B091B603C82AD92AEA2AFB2ACFE1D0E02C
:104D0000D701C6010C2E04C0B695A7959795879537
:104D10000A94D2F780FF06C0B8018C2F0E942F0A98
:104D2000019721F4219760F780E001C08C2FDF917B
:104D3000CF911F910F91FF90EF90DF90CF9008954A
:104D4000CF93DF93EC010E946126BE010E942F0ADF
:104D5000DF91CF910895CB010E94A0260895209164
:104D60001D0230911E02F90132969FEF40E05191F1
:104D7000581789F09F3F19F4511101C0942F4F5FCC
:104D80004630A9F79F3F39F0F901E90FF11D97FD72
:104D9000FA9582830895089520911D0230911E0294
:104DA000F9013296285F3F4F9081981301C010821D
:104DB0003196E217F307C1F7089581E090E0E091A2
:104DC0001D02F0911E02E80FF91F10820196883033
:104DD0009105A9F708959091C603892B8093C60386
:104DE000089580959091C60389238093C603089502
:104DF0001092C60308959091C503892B8093C50333
:104E0000089580959091C50389238093C5030895E3
:104E10001092C50308959091C403892B8093C40315
:104E2000089580959091C40389238093C4030895C5
:104E30001092C40308958093BB0308951092BB039E
:104E4000089580911D0290911E02FC0131969C01F3
:104E5000285F3F4F80E0919191118F5FE217F30738
:104E6000D1F70895E0911D02F0911E028091C603D2
:104E70008083E0911D02F0911E0290818091C50314
:104E8000892B8083E0911D02F0911E029081809118
:104E9000C403892B80838091BB03882361F0E09158
:104EA0001D02F0911E029081892B80830E94212790
:104EB00081111092BB0380911D0290911E020C94EF
:104EC0005B1B8091E803843039F11092C80320E421
:104ED00088E190E00FB6F894A895809360000FBE2B
:104EE0002093600080E00E94D20580E00E940A0BBF
:104EF00083B7817F846083BF83B7816083BF7894E9
:104F0000889583B78E7F83BF88E10FB6F89480932E
:104F10006000109260000FBE089508950895CF9329
:104F200080E00E94D2050E948D270E94AD0C0E9455
:104F30008E27C0E08C2F0E94E60D892B29F4CF5FCD
:104F4000C530C1F780E001C081E0CF9108950E9493
:104F50006C2180E00E94D2050E94092D0E944F1B07
:104F60000C940A0B1F920F920FB60F9211248F937D
:104F70009F93AF93BF938091C803811113C0809119
:104F8000C9039091CA03A091CB03B091CC03419681
:104F9000A11DB11D8093C9039093CA03A093CB03B5
:104FA000B093CC03BF91AF919F918F910F900FBEA3
:104FB0000F901F90189582E084BD93E095BD9AEF05
:104FC00097BD80936E0008952FB7F8948091C90320
:104FD0009091CA03A091CB03B091CC032FBF089549
:104FE000CF92DF92EF92FF920F931F932FB7F89417
:104FF0004091C9035091CA036091CB037091CC03D7
:105000002FBF6A017B01EE24FF248C0120E030E0F9
:10501000C016D106E206F30610F4415051099A0178
:10502000281B390BC9011F910F91FF90EF90DF9062
:10503000CF9008951F920F920FB60F9211248F9365
:105040009F93AF93BF938091C9039091CA03A0919E
:10505000CB03B091CC030196A11DB11D8093C90370
:105060009093CA03A093CB03B093CC03BF91AF91AD
:105070009F918F910F900FBE0F901F9018950E94D7
:105080004C18F8942FEF87EA91E621508040904029
:10509000E1F700C0000087E090EBDC018093F303B0
:1050A0009093F403A093F503B093F6039CE088E19A
:1050B0000FB6F894A895809360000FBE909360009F
:1050C000FFCF0E949B28811102C00E9477280E9476
:1050D000A6288093C7030E94B3288093F1030E94FF
:1050E000AA28682F70E080E090E00C9428256DEEEF
:1050F0007EEF80E090E00E94BC3160E082E090E0D2
:105100000E94AA3160E083E090E00E94AA3160E052
:1051100084E090E00E94AA3160E085E090E00E9487
:10512000AA3160E086E090E00E94AA316FEF87E04C
:1051300090E00C94AA3180E090E00E94A43121E03C
:105140008D3E9E4F09F020E0822F089582E090E08E
:105150000C949C3183E090E00C949C31682F83E0A8
:1051600090E00C94AA3184E090E00C949C31682F7C
:1051700084E090E00C94AA3186E090E00C949C319D
:10518000682F86E090E00C94AA3187E090E00C94C0
:105190009C31682F87E090E00C94AA318091CF0376
:1051A00080FF0BC06091220285E0689FB00111244E
:1051B00075956795759567952BC081FF09C06091BE
:1051C000220285E0689FB00111247595679520C083
:1051D00082FF07C06091220285E0689FB001112420
:1051E00017C09091D0039923D1F0609121029617B6
:1051F00088F72091220285E0289F90011124929F38
:10520000A001939F500D112470E0CA010E948231C9
:105210006038710540F46115710539F002C065E030
:1052200070E0862F08958FE7089581E008958091BA
:10523000CF0380FF08C06091200270E075956795EC
:105240007595679521C081FF06C06091200270E0CE
:105250007595679519C082FF04C06091200270E0C7
:1052600010C09091D0039923C1F060911F0296174E
:10527000A0F780912002899FC001112470E00E9454
:1052800082316038710528F46115710521F0862F8F
:1052900008958FE7089581E0089561E070E0F4CF0C
:1052A000803F21F40E94CE28819504C0813F29F4DB
:1052B0000E94CE288093D3030895823F21F40E9458
:1052C000CE28819504C0833F29F40E94CE28809384
:1052D000D2030895893F19F40E94172905C08A3F17
:1052E00031F40E94172981958093D40308958B3F50
:1052F00021F40E941729819504C08C3F29F40E9453
:1053000017298093D5030895843F21F48091D10318
:10531000816017C0853F21F48091D103826011C064
:10532000863F21F48091D10384600BC0873F21F434
:105330008091D103886005C0883F31F48091D1030A
:1053400080618093D10308958D3F21F48091CF0334
:1053500081600BC08E3F21F48091CF03826005C035
:105360008F3F29F48091CF0384608093CF03089509
:10537000803F39F48091D30387FF6CC01092D30330
:1053800069C0813F29F48091D3031816BCF362C031
:105390009091D203823F29F497FF5CC01092D20310
:1053A00059C0833F19F41916CCF354C0893F41F416
:1053B0008091D40318160CF04DC01092D4034AC04B
:1053C0008A3F29F48091D40387FF44C0F6CF8B3FF6
:1053D00039F48091D50387FF3DC01092D5033AC0C0
:1053E0008C3F29F48091D5031816BCF333C0843F59
:1053F00021F48091D1038E7F17C0853F21F48091E5
:10540000D1038D7F11C0863F21F48091D1038B7F22
:105410000BC0873F21F48091D103877F05C0883F6F
:1054200031F48091D1038F7E8093D10313C08D3FDF
:1054300021F48091CF038E7F0BC08E3F21F48091A9
:10544000CF038D7F05C08F3F29F48091CF038B7FE1
:105450008093CF038091D20381110EC08091D3033A
:1054600081110AC08091D403811106C08091D503B7
:10547000811102C01092D003089581ED93E00E9443
:10548000661B0E94E4279093CE038093CD0308957A
:105490001F93CF93DF938091CD039091CE030E9411
:1054A000F027AC019091D003992321F020912302A1
:1054B00030E006C0209124028AE0289F9001112448
:1054C0004217530708F486C08091D203C091D303DA
:1054D000D091D4031091D503811107C0C11176C0BA
:1054E000D11174C0111172C075C09F3F19F09F5F38
:1054F0009093D003181624F40E94CE288093D203F0
:105500008091D20387FF05C00E94CE2881958093A9
:10551000D2031C1624F40E94CE288093D3038091DA
:10552000D30387FF05C00E94CE2881958093D303C3
:105530006091D203662339F1C091D303CC2319F1D2
:10554000772767FD7095872F972F0E94A42E23E35E
:1055500033E343E35FE30E94B42F0E94712E609314
:10556000D2036C2F772767FD7095872F972F0E94A6
:10557000A42E23E333E343E35FE30E94B42F0E94AE
:10558000712E6093D3031D1624F40E941729809373
:10559000D4038091D40387FF05C00E941729819509
:1055A0008093D403111624F40E9417298093D50305
:1055B0008091D50387FF05C00E94172981958093AC
:1055C000D503DF91CF911F910C943D2A9F3F09F0A5
:1055D0008ECF96CFDF91CF911F910895E1EDF3E04B
:1055E00085E0DF011D928A95E9F71092D0031092B1
:1055F000CF030895833081F128F4813059F082304F
:10560000D1F00895853009F449C0B8F1863009F425
:1056100056C0089580912402262F30E0280F311DB6
:105620002F3F310524F4680F6093240208958FEF13
:1056300080932402089580912302262F30E0280FC2
:10564000311D2F3F310524F4680F60932302089524
:105650008FEF80932302089580912202262F30E05D
:10566000280F311D2F3F310524F4680F609322026B
:1056700008958FEF80932202089580912102262FB2
:1056800030E0280F311D2F3F310524F4680F60935F
:10569000210208958FEF80932102089580912002C6
:1056A000262F30E0280F311D2F3F310524F4680FDD
:1056B0006093200208958FEF8093200208958091D7
:1056C0001F02262F30E0280F311D2F3F310524F413
:1056D000680F60931F0208958FEF80931F02089553
:1056E000833011F128F4813049F0823091F008952F
:1056F000853081F120F18630C1F108958091240236
:10570000681720F4861B80932402089510922402C7
:10571000089580912302681720F4861B809323024A
:10572000089510922302089580912202681720F4B0
:10573000861B809322020895109222020895809180
:105740002102681720F4861B80932102089510928D
:105750002102089580912002681720F4861B80930F
:105760002002089510922002089580911F02681768
:1057700020F4861B80931F02089510921F02089543
:105780000F931F938732D8F58E3108F087C08E3083
:1057900009F471C098F4873009F45BC08B3009F4C8
:1057A00091C0863009F095C08091C703817F8E7FBC
:1057B0008093C70381E08093D7038CC0863109F4BE
:1057C00081C068F4803109F084C08091C70383FBF5
:1057D000222720F991E0922790FB83F955C0893167
:1057E00009F470C08B3109F074C08091C70381FB4C
:1057F000222720F991E0922790FB81F945C0883358
:1058000009F460C050F4893209F45EC0853309F4AC
:105810005BC0873209F458C05CC0833409F454C0BB
:1058200028F48A3308F455C0895339C0883409F004
:1058300050C00E946C210E94B2070FEF13ED20E3CD
:10584000015010402040E1F700C000000E943F28B6
:1058500039C09091C703892F8095817080FB90F9A2
:1058600029F0966098609093C70334C0997F977F22
:105870009093C70327C08091C70382FB222720F99A
:1058800091E0922790FB82F98093C7039923D1F08E
:105890008091C70381608093C70314C08D5141E09C
:1058A00050E060E070E08A019B0104C0000F111F0E
:1058B000221F331F8A95D2F7C901B8010E942825FB
:1058C0000E946C2181E006C061E070E080E090E021
:1058D000F5CF80E01F910F91089580E0089580E05A
:1058E0000895CF93C82F8091D703813069F018F0C5
:1058F0008230C9F184C0E0911D02F0911E028081C6
:10590000823209F07EC007C0E0911D02F0911E02B4
:105910008081823261F48C2F0E946D2C811104C031
:105920008C2F0E94C02B1DC081E090E01AC08C2FEC
:105930000E946F2C811114C0C43179F048F4CB302F
:1059400079F0C03109F061C082E08093D70308C0CC
:10595000C93219F0C83321F058C01092D70355C08E
:1059600081E0817054C0C93291F120F5C43179F1E0
:10597000B0F4C73009F047C08EE18093240282E37F
:10598000809323028AE08093220284E180932102A3
:1059900088E08093200288E280931F0234C0CE51B9
:1059A000C63088F5EC2FF0E0E451FD4F8081809304
:1059B000D60329C0CE34E9F020F4CB3421F56AE0D7
:1059C00013C0C13579F0C235F1F461E00DC08091AA
:1059D000D603882319F01092D60315C081E0809376
:1059E000D70315C061E006C08091D6030E94FA2A51
:1059F0000AC06AE08091D6030E94702B04C0109206
:105A0000D70380E004C081E002C080E0AACFCF913C
:105A100008950E949B28811102C00E9477280E944D
:105A2000BC288093F20380FF02C0869501C080E00D
:105A30000C94D2058091F203982F9695292F30E08F
:105A4000233031054CF49F5F990F8170892B816061
:105A50008093F2030E94C0288091F20386950C94F3
:105A6000D2058091F203982F969591F09158990F55
:105A70008170892B8093F2038E7F91E009F490E08E
:105A80008091F20390FB80F98093F2030E94C0287A
:105A90008091F20386950C94D2058091F203982FA1
:105AA000909590FB80F98093F2030E94C02880912A
:105AB000F20380FF02C0869501C080E00C94D205FD
:105AC0009091F203892F86958F5F8F779170843044
:105AD00028F4880F892B8093F20302C09093F2037D
:105AE0008091F2038E7F91E009F490E08091F203BF
:105AF00090FB80F98093F2030E94C0288091F2030A
:105B000086950C94D2052091F203922F96958927C1
:105B1000982F990F822F8170892B8093F2038E7FAB
:105B200091E009F490E08091F20390FB80F980937A
:105B3000F2030E94C0288091F20386950C94D2054E
:105B40005058BB27AA270ED0D1C1C2D130F0C7D13F
:105B500020F031F49F3F11F41EF4B7C10EF4E0952C
:105B6000E7FB9FC1E92FD3D180F3BA176207730710
:105B70008407950718F071F49EF5EBC10EF4E095DB
:105B80000B2EBA2FA02D0B01B90190010C01CA01F7
:105B9000A0011124FF27591B99F0593F50F4503EA2
:105BA00068F11A16F040A22F232F342F4427585F94
:105BB000F3CF469537952795A795F0405395C9F7AC
:105BC0007EF41F16BA0B620B730B840BBAF0915064
:105BD000A1F0FF0FBB1F661F771F881FC2F70EC003
:105BE000BA0F621F731F841F48F4879577956795D6
:105BF000B795F7959E3F08F0B3CF9395880F08F0BF
:105C00009927EE0F97958795089527D108F481E09D
:105C100008950CD06BC163D140F05AD130F021F41B
:105C20005F3F19F03EC1511195C14FC170D198F33A
:105C30009923C9F35523B1F3951B550BBB27AA270D
:105C400062177307840738F09F5F5F4F220F331F7F
:105C5000441FAA1FA9F333D00E2E3AF0E0E830D04B
:105C600091505040E695001CCAF729D0FE2F27D04E
:105C7000660F771F881FBB1F261737074807AB071C
:105C8000B0E809F0BB0B802DBF01FF2793585F4F91
:105C90002AF09E3F510568F004C15CC15F3FECF300
:105CA000983EDCF3869577956795B795F7959F5F56
:105CB000C9F7880F911D9695879597F90895E1E0AA
:105CC000660F771F881FBB1F621773078407BA0709
:105CD00020F0621B730B840BBA0BEE1F88F7E09564
:105CE000089504D06894B11135C1089518D188F091
:105CF0009F5790F0B92F9927B751A0F0D1F0660FB8
:105D0000771F881F991F1AF0BA95C9F712C0B130D2
:105D100081F01FD1B1E008951CC1672F782F88272B
:105D2000B85F39F0B93FCCF3869577956795B39511
:105D3000D9F73EF490958095709561957F4F8F4F80
:105D40009F4F0895E89409C097FB3EF49095809585
:105D5000709561957F4F8F4F9F4F9923A9F0F92F31
:105D600096E9BB279395F695879577956795B795AF
:105D7000F111F8CFFAF4BB0F11F460FF1BC06F5F95
:105D80007F4F8F4F9F4F16C0882311F096E911C0A7
:105D9000772321F09EE8872F762F05C0662371F0C8
:105DA00096E8862F70E060E02AF09A95660F771FDC
:105DB000881FDAF7880F9695879597F9089588D008
:105DC00018F011F08CD038F480C0C4C0E92F9FD0F7
:105DD000B0F35523C9F3E7FB6217730784079507F0
:105DE000A8F199F3E92FFF2788232AF03197660F4E
:105DF000771F881FDAF7952F5527442332F09150EB
:105E00005040220F331F441FD2F7BB27E91BF50B6D
:105E1000621B730B840BB109C1F222F4620F731F72
:105E2000841FB11D31972AF0660F771F881FBB1F93
:105E3000EFCF915050405AF041F0882332F0660F76
:105E4000771F881F91505040C1F7939530C08695B9
:105E5000779567959F5FD9F7F8CF990F0008550F91
:105E6000AA0BE0E8FEEF16161706E807F907C0F0E0
:105E700012161306E407F50798F0621B730B840BE8
:105E8000950B39F40A2661F0232B242B252B21F4C2
:105E900008950A2609F4A140A6958FEF811D811D62
:105EA000089597F99F6780E870E060E008959F3F4C
:105EB00031F0915020F4879577956795B795880FC5
:105EC000911D9695879597F908959FEF80EC089519
:105ED00000240A94161617061806090608950024C9
:105EE0000A9412161306140605060895092E039443
:105EF000000C11F4882352F0BB0F40F4BF2B11F4B7
:105F000060FF04C06F5F7F4F8F4F9F4F089557FD15
:105F10009058440F551F59F05F3F71F04795880F17
:105F200097FB991F61F09F3F79F0879508951216AE
:105F300013061406551FF2CF4695F1DF08C016165A
:105F400017061806991FF1CF86957105610508940B
:105F50000895E894BB2766277727CB0197F9089522
:105F60007CDF08F48FEF08950BD0C0CFB1DF28F0AD
:105F7000B6DF18F0952309F094CFA7CF1124EACF0C
:105F8000C6DFA0F3959FD1F3950F50E0551F629F98
:105F9000F001729FBB27F00DB11D639FAA27F00D82
:105FA000B11DAA1F649F6627B00DA11D661F829FA9
:105FB0002227B00DA11D621F739FB00DA11D621F8E
:105FC000839FA00D611D221F749F3327A00D611DAB
:105FD000231F849F600D211D822F762F6A2F11248D
:105FE0009F5750408AF0E1F088234AF0EE0FFF1FE0
:105FF000BB1F661F771F881F91505040A9F79E3F17
:10600000510570F04ECFA6CF5F3FECF3983EDCF326
:10601000869577956795B795F795E7959F5FC1F753
:10602000FE2B880F911D9695879597F90895FA0193
:10603000EE0FFF1F30962105310599F161157105AD
:1060400061F48038BFE39B0749F16894903881057B
:1060500061F08038BFEF9B0741F0992342F5FF3F85
:10606000E1053105210511F1E8940894E795D9017E
:10607000AA2329F4AB2FBE2FF85FD0F310C0FF5F27
:1060800070F4A695E0F7F73950F019F0FF3A38F4BC
:106090009F779F930CD00F9007FC905808953EF087
:1060A00014CF60E070E080E89FE308954FE79F77AA
:1060B0005F934F933F932F939ED02F913F914F919A
:1060C0005F9152DF05C019F40EF0EBCE42CFFDCE4A
:1060D00026DFC8F39638C0F707F80F92E8942BE351
:1060E0003AEA48EB5FE74EDF0F920F920F924DB7FF
:1060F0005EB70F92C0D0E8EFF0E016D04F915F91FD
:10610000EF91FF91E595EE1FFF1F49F0FE57E06804
:106110004427EE0F441FFA95E1F74195550B32D015
:106120000F9007FE26C00895DF93CF931F930F9320
:10613000FF92EF92DF927B018C01689405C0DA2E0A
:10614000EF011EDFFE01E894A5912591359145915F
:106150005591AEF3EF0106DDFE019701A801DA9437
:1061600079F7DF90EF90FF900F911F91CF91DF9122
:1061700008959B01AC0160E070E080E89FE349CDA9
:1061800090CE95CECCDEE8F39923D9F3940F511D30
:10619000BBF39150504094F059F0882332F0660FD1
:1061A000771F881F91505040C1F79E3F510544F71B
:1061B000880F911D9695879597F908955F3FACF0EC
:1061C000983E9CF0BB27869577956795B79508F420
:1061D000B1609395C1F7BB0F58F711F460FFE8CF9A
:1061E0006F5F7F4F8F4F9F4FE3CFB4CE0EF05FCEE8
:1061F0006CCE689456CE93DEC8F39923D1F3C6F3E0
:10620000DF93CF931F930F93FF92C92FDD2788232E
:106210002AF02197660F771F881FDAF720E030E019
:1062200040E85FEB9FE3883920F0803E30F0219614
:106230008F7787DCE0E2F1E003C083DCEDE4F1E09E
:1062400073DF8B01BE01EC01FB2E6F577109759551
:10625000771F880B990B78DD28E132E741E35FE394
:106260008FDEAF2D9801AE01FF900F911F91CF915E
:10627000DF9178DC3BCEFA01DC01AA0FBB1F9B014A
:10628000AC01BF5728F422273327442750781FC07A
:10629000B75188F4AB2F0024469537952795011CFC
:1062A000A395D2F3002069F0220F331F441FB3954A
:1062B000DAF30DD045CC61307105A0E88A07B94604
:1062C00030F49B01AC0166277727882790783096B9
:1062D00021F020833183428353830895AA1BBB1B83
:1062E00051E107C0AA1FBB1FA617B70710F0A61BD6
:1062F000B70B881F991F5A95A9F780959095BC01F7
:10630000CD01089597FB072E16F4009407D077FD72
:1063100009D00E946E3107FC05D03EF4909581951E
:106320009F4F0895709561957F4F0895EE0FFF1F61
:106330000590F491E02D0994F999FECF92BD81BDAD
:10634000F89A992780B50895A8E1B0E042E050E0BE
:106350000C94C431262FF999FECF92BD81BDF89AD5
:10636000019700B4021639F01FBA20BD0FB6F89499
:10637000FA9AF99A0FBE08950196272F0E94AB3121
:106380000C94AA31DC01CB01FC01F999FECF06C0C7
:10639000F2BDE1BDF89A319600B40D9241505040E3
:0863A000B8F70895F894FFCF4F
:1063A8000C52D02445000000410000DC44000000ED
:1063B8004152D0A4440000404100005C4400000069
:1063C8004148F17644000000415C978A440000008F
:1063D800411FD592440000004152D0A4440000005F
:1063E800415CFFB844000000410AA7CF4400000008
:1063F800410000DC44000000410AA7CF440000002F
:10640800410000DC44000000410000000000008062
:106418004052D024450000404100000000000080A8
:10642800400AA74F45000040410AA7CF440000009A
:10643800410000DC44000000410000000000008032
:106448004052D024450000004100000000000080B8
:10645800405CFF384500000041000000000000805B
:106468004052D02445000000410AA7CF4400000054
:10647800410000DC440000004100000000000080F2
:106488004052D024450000804110F176440000A01D
:106498004112F1F6440000004141909B440000A0E5
:1064A8004112F1F64400000041050000003F0000E1
:1064B800C8427B140915E614B2147E1401BC0328E3
:1064C80008140A321E000002000400050007000933
:1064D800000B000C000E001000110013001500172F
:1064E8000018001A001C001D001F002100230024B2
:1064F800002600280029002B002D002F0030003234
:106508000034003500370039003B004200450025C3
:106518000026004300610060002000370064006529
:1065280000660067004400460024004700314980A7
:106538003F5D8B803FF8BF803FCAE1803F73ED80AD
:106548003FCAE1803FF8BF803F5D8B803F31498083
:106558003F0000803FF16D7F3F75EA7E3F4C827EB1
:106568003F833F7E3F84287E3F833F7E3F4C827E31
:106578003F75EA7E3FF16D7F3F0000803F3F4D361B
:10658800B90A6C0A360AE209FB09140A0102030473
:06659800050607080900DA
:00000001FF
